:040000007CEF25F07C
:1000080000C016F001C015F0E1CF17F0E2CF18F0EC
:100018009DAA75D09EAA73D0AECF4EF1ABA40ED0D8
:10002800AB9E010E2224006E000E2320016E00C03C
:1000380022F001C023F0AB8E01014E6BABA20ED0B3
:100048000101AB98010E2024006E000E2120016EE4
:1000580000C020F001C021F0AB884E6B01014E5169
:100068000D0A3BE08B0E3724E16E000E3820E26E5D
:100078004EC1E6FF37C039F038C03AF0010E3724D8
:10008800006E000E3820016E00C037F001C038F055
:10009800800E006E800E3818005C02E137504F0861
:1000A80019E2020E2C6E000E2D6E9D9A010E375C21
:1000B800006E000E3858016E8B0E0024E16E000EA3
:1000C8000120E26EE66A37C039F038C03AF0376A84
:1000D800386A02D02C6A2D6A11D08B0E3724E16E53
:1000E800000E3820E26EE66A010E2C6E000E2D6EB0
:1000F80037C039F038C03AF0376A386A9E9A16C065
:1001080000F015C001F017C0E1FF18C0E2FF1100B0
:10011800EACDEEFDEBCDEFFDECCDEAFDEDCDEBFD4F
:0A012800EECDECFDEFCDEDFD120071
:10013200EACDC9FFC7B002D00000FCD7C9CF00F09A
:020142001200A9
:100144008B928B94E7CD00F0016A00C0EAFDEFDFEB
:10015400FF0E0D01E615EA6FEADF00008B82E9CDA0
:1001640000F0016A00C0EAFDE2DFFF0E0D01E815B0
:08017400EA6FDDDF8B8412004D
:10017C0041D04DD00D01E851975DE86FE951985988
:10018C00E96F010EE85F000EE95BE6CDEAFDE7CD15
:10019C00EBFDE8CDECFDE9CDEDFDB8DF38D00D0180
:1001AC00E651335CE66FE7513458E76F010EE65FBA
:1001BC00000EE75BE851975DE86FE9519859E96FDC
:1001CC00010EE85F000EE95B22D00D01E651335CB5
:1001DC00E66FE7513458E76F010EE65F000EE75B00
:1001EC00E6CDEAFDE7CDEBFDE8CDECFDE9CDEDFD8F
:1001FC008DDF0DD001015751000ABBE05751010AA8
:10020C00B9E05751020ACBE05751030ADEE0120065
:10021C008B928B94E6CDEAFD86DFE7CDEAFD83DF9A
:04022C008B841200AD
:0E0230008B928B94E6CDEAFD7CDF8B8412006E
:10023E00DECDE6FDDFCDE7FDE0CDE8FDE1CDE9FD6C
:10024E0096DFE2CDE6FDE3CDE7FDE4CDE8FDE5CDBD
:10025E00E9FD8DDF800E0D01E319006E800EDF19B2
:10026E00005C02E1DE51E25D09E2DECDEAFDDFCDAA
:10027E00EBFDE2CDECFDE3CDEDFD47DF800EE519A4
:10028E00006E800EE119005C02E1E051E45D09E2CE
:10029E00E0CDEAFDE1CDEBFDE4CDECFDE5CDEDFDF0
:1002AE0034DF360EE66F000EE76FE2CDE8FDE3CDEC
:1002BE00E9FD41DF370E0D01E66F000EE76FDECD73
:1002CE00E8FDDFCDE9FD37DF380E0D01E66F000EDC
:1002DE00E76FE4CDE8FDE5CDE9FD2DDF390E0D012B
:1002EE00E66F000EE76FE0CDE8FDE1CDE9FD23DF1F
:1002FE00200E0D01E66F000EE76FDECDE8FDDFCDBF
:10030E00E9FD19DF210E0D01E66F000EE76FE0CD5E
:10031E00E8FDE1CDE9FD0FDF220E0D01E66F81DF75
:0C032E000D01E66B220EE76F72DF12007B
:10033A008B828B94DECDEAFDF7DEDFCDEAFDF4DEBB
:04034A008B8412008E
:08034E000AAE029E000E12002F
:100356000B840BAEB6EF01F0010E036E026A016A62
:0A036600006A0A360232FF0E120090
:0E037000026A016A006A086A036A000E12003F
:10037E000B820BAEC9EF01F00368026801680068DA
:08038E000A360232FF0E1200D4
:0E039600ACB202D00000FCD7D6CDADFF1200F5
:1003A400086A080E0C6E003408360450085ED8B093
:0E03B40002D00826D89000360C2EF5D7120085
:1003C20034500D01D75D02E13350D65D07E29851FA
:1003D200D95D02E19751D85D01E201D026D0D6CD98
:1003E200DEFDD7CDDFFDD8CDE0FDD9CDE1FD010E9B
:1003F200D625E26F000ED721E36F010ED825E46FF8
:10040200000ED921E56F1ADFD6CDE6FDD7CDE7FD87
:10041200D8CDE8FDD9CDE9FDB0DEDBCD00F0016A33
:0C04220000C0DEFDDACDDFFD87DF120038
:10042E00000E0D01D71902E1000ED61902E1006A85
:10043E002ED0000EDB1902E1000EDA1902E1006A7D
:10044E0026D0D751DB1902E1DA51D61902E1006A42
:10045E001ED0D851D625016ED951D721026E025029
:10046E00DB1902E1DA51011803E1010E006E0FD023
:10047E00DC51DA25016EDD51DB21026E0250D719F7
:10048E0002E1D651011803E1020E006E00D01200F7
:10049E000B6A0A6A096A00500402F4CF09F0F3CF1E
:1004AE0008F001500502F4CF0BF0F3CF0AF0005024
:1004BE000502F3500926F4500A22E86A0B22015075
:1004CE000402F3500926F4500A22E86A0B2208C0EF
:1004DE0000F009C001F00AC002F00BC003F01200D8
:1004EE000134083609360450085E0550D8A0053C84
:1004FE00095E003601360F0E0C6E013408360936D1
:10050E00045000A006D0085E0550D8A0053C095E38
:10051E0005D008260550D8B0053C09260036013610
:10052E000C2EEBD700B006D0045008260550D8B0DC
:08053E00053C09260000120033
:100546000CB0E5EF02F00CA28BEF03F00E6A000E82
:100556000264FCEF02F0F00E0214D8A4C7EF02F01A
:10056600023A01380F0B02260138F00B016E0038F3
:100576000F0B01260038F00B006E08380F0B002613
:100586000838F00B086E0E84D89002BEE0EF02F039
:1005960008360036013602360E2A02BEE0EF02F0B9
:1005A60008360036013602360E2A02BEE0EF02F0A9
:1005B60008360036013602360E2A0E50036481EFE5
:1005C60003F0035E0BBC08AE86EF03F0D880800E06
:1005D60008640030000E002201220222D8A086EF15
:1005E60003F0023201320032034A8BEF03F086EF4A
:1005F60003F001C002F000C001F008C000F0086A74
:10060600000E0E86026433EF03F0F00E0214D8A437
:100616001BEF03F0023A01380F0B02260138F00BEC
:10062600016E00380F0B01260038F00B006E0E84A9
:10063600D89002BEE0EF02F00036013602360E2AEE
:1006460002BEE0EF02F00036013602360E2A02BE86
:10065600E0EF02F00036013602360E2AE0EF02F035
:1006660001C002F000C001F0006A000E0E960E886E
:10067600026460EF03F0F00E0214D8A44BEF03F00F
:10068600023A01380F0B02260138F00B016E0E8478
:10069600D89002BEE0EF02F0013602360E2A02BE04
:1006A600E0EF02F0013602360E2A02BEE0EF02F05B
:1006B600013602360E2AE0EF02F001C002F0016AAE
:1006C600000E0E86026490EF03F0F00E0214D8A41A
:1006D6006FEF03F0023A0E84D89002BEE0EF02F00C
:1006E60002360E2A02BEE0EF02F002360E2A02BEE3
:1006F600E0EF02F002360E2AE0EF02F0010E0C6E79
:1007060027DE93EF03F0020E0C6E1EDE93EF03F06E
:10071600040E0C6E31DE93EF03F0080E0C6E25DE30
:020726001200BF
:10072800C6CDF6FFC7CDF7FFC8CDF8FF0900F5CF56
:1007380000F0005211E0C6CDF6FFC7CDF7FFC8CDD7
:10074800F8FF0900F5CFD6FD22DE010E0D01C62700
:0A075800000EC723C823E4D71200E7
:10076200025006180E6E086A096A0B6A0350076483
:10077200A4EF04F006500A6E068E028E03500B6E32
:100782000750036E000E0B64F4EF03F00B50075E8C
:10079200D8B495EF04F0070E076463EF04F0075E28
:1007A20000C008F001C000F002C001F0026A074E6A
:1007B20095EF04F0076438EF04F0075E00C008F01C
:1007C20001C000F0016A074E95EF04F0076416EFCE
:1007D20004F0075E00C008F0006A074E95EF04F0CF
:1007E2000764FDEF03F00AC002F005C001F004C087
:1007F20000F0086ABEEF05F0030E076408EF04F08C
:10080200075E08380F0B086E074E95EF04F0D8907C
:100812000832074E95EF04F0D8900832074E95EF54
:1008220004F0D890083295EF04F0030E076427EF26
:1008320004F0075E08380F0B086E0038F00B08262C
:1008420000380F0B006E074E95EF04F0D89000327F
:100852000832074E95EF04F0D89000320832074E66
:1008620095EF04F0D8900032083295EF04F0030EB1
:1008720007644FEF04F0075E08380F0B086E00386C
:10088200F00B082600380F0B006E0138F00B002623
:1008920001380F0B016E074E95EF04F0D89001322C
:1008A20000320832074E95EF04F0D8900132003240
:1008B2000832074E95EF04F0D89001320032083228
:1008C20095EF04F0030E076480EF04F0075E08382A
:1008D2000F0B086E0038F00B082600380F0B006E65
:1008E2000138F00B002601380F0B016E0238F00BB5
:1008F200012602380F0B026E074E95EF04F0D890D6
:100902000232013200320832074E95EF04F0D890DD
:100912000232013200320832074E95EF04F0D890CD
:100922000232013200320832096A000E0EAE89EF3D
:1009320005F0081E001E011E021E082A00220122C6
:10094200022289EF05F00750D8A4AAEF04F0BEEF07
:1009520005F0096A02C00AF0028E068E0750035C97
:10096200076ED8B47CEF05F0070E07644AEF05F076
:10097200075E0450096E0550046E0650056E066A45
:10098200074E7CEF05F0070E07641FEF05F0075EC8
:100992000450096E0550046E056A074E7CEF05F09F
:1009A200070E0764FDEF04F0075E0450096E046A47
:1009B200074E7CEF05F0070E0764E4EF04F00AC06F
:1009C20002F0BEEF05F0030E0764EFEF04F0075EDE
:1009D20009380F0B096E074E7CEF05F0D8900932EB
:1009E200074E7CEF05F0D8900932074E7CEF05F0F8
:1009F200D89009327CEF05F0030E07640EEF05F084
:100A0200075E09380F0B096E0438F00B092604380B
:100A12000F0B046E074E7CEF05F0D89004320932BA
:100A2200074E7CEF05F0D89004320932074E7CEF76
:100A320005F0D890043209327CEF05F0030E07640A
:100A420036EF05F0075E09380F0B096E0438F00B1C
:100A5200092604380F0B046E0538F00B04260538FE
:100A62000F0B056E074E7CEF05F0D890053204326D
:100A72000932074E7CEF05F0D89005320432093274
:100A8200074E7CEF05F0D8900532043209327CEF34
:100A920005F0030E076467EF05F0075E09380F0BD8
:100AA200096E0438F00B092604380F0B046E053862
:100AB200F00B042605380F0B056E0638F00B0526E1
:100AC20006380F0B066E074E7CEF05F0D890063203
:100AD200053204320932074E7CEF05F0D890063217
:100AE200053204320932074E7CEF05F0D890063207
:100AF200053204320932086A000E0EAE89EF05F0A3
:100B0200091E041E051E061E092A042205220622AB
:100B120009500826045000220550012206500222E4
:100B22000EBEA0EF05F0D8A0AFEF05F00232013201
:100B320000320832033EAFEF05F0B9EF05F0D8B04E
:100B4200B4EF05F0000E081E001E011E021E082A48
:100B52000022012202220A7EB4EF05F0010E0C6E81
:100B6200F1DCC0EF05F0020E0C6EECDCC0EF05F01C
:100B7200040E0C6E03DCC0EF05F0000E0C6E1200CA
:080B82000B6A0B86FF0E120046
:100B8A000D01C96BC6CDE9FFC7CDEAFFEECFC8FD9F
:100B9A00C851000A0FE0C8CDD6FDCBEC01F00D011B
:100BAA00C92BC951C625E96E000EC721EA6EEECFE0
:060BBA00C8FDEED7120099
:100BC0000B800BAEECEF05F0026A0AAEFF0E026E70
:0C0BD000016E006E0A360232FF0E1200A9
:100BDC000D01C96B030EC95D0AE2C951C725E16E4F
:100BEC00000EC821E26E200EE66EC92BF3D7C95158
:100BFC00C725E16E000EC821E26EE66AC907C9512D
:100C0C00C725CA6F000EC821CB6F0A0E046EC6CD65
:100C1C0000F0D2EC01F008C000F0300E0026CACD76
:100C2C00E1FFCBCDE2FF00C0E6FF0A0E046EC6CD9D
:100C3C0000F0D2EC01F000C0C6FD0050000A01E14A
:080C4C0002D0C907DCD7120039
:100C54000C6A0E6A0250D8A443EF06F001C002F0F9
:100C640000C001F0006A0E860250D8A443EF06F0DB
:100C740001C002F0016A0E960E880250D8B455EFF6
:100C840006F00E50035ED8A4D8A05BEF06F0D8900F
:100C940002BE61EF06F0003601360236032E4AEF3B
:100CA40006F05BEF06F0010E0C6EB8EC01F065EF98
:100CB40006F0020E0C6EABEC01F065EF06F0040ECC
:080CC4000C6EA7EC01F0120018
:100CCC00086A096A100E0C6E013408360936045095
:100CDC00085E0550D8A0053C095ED8B007D004507A
:100CEC0008260550D8B0053C0926D89000360136A8
:060CFC000C2EEAD71200E5
:100D02000D01C86BC96B0001E45305E0C8CD00F0CA
:100D1200C9CD01F020D10D01CA6B800E006E800E8C
:100D2200000A005C02E1140ECA5DD8B010D1040EB4
:100D3200006E000E016ECACD04F0000E056E4FEC7F
:100D420002F0F50E0026000E012200C0E9FF01C0EC
:100D5200EAFFEECF01F0EECF02F0000E006E02507D
:100D6200005C02E101500008D8B0EED00D01040E83
:100D7200006E000E016ECACD04F0000E056E4FEC3F
:100D820002F0F50E0026000E0122020E0024E96E8A
:100D9200000E0120EA6EEECF01F0EECF02F0C75155
:100DA200025C02E1C651015CD8A0CED0040E006EF6
:100DB200000E016ECACD04F0000E056E4FEC02F07B
:100DC200F50E0026000E012200C0E9FF01C0EAFF75
:100DD200EECFC8FDEECFC9FD040E006E000E016E0F
:100DE200CACD04F0000E056E4FEC02F0F50E00269F
:100DF200000E0122020E0024E96E000E0120EA6EAE
:100E0200EECF01F0EECF02F00250C75D02E10150D9
:100E1200C65D69E2040E006E000E016ECACD04F0DA
:100E2200000E056E4FEC02F0F50E0026000E0122B8
:100E320000C0CBFD01C0CCFD040E006E000E016EA1
:100E4200CACD04F0000E056E4FEC02F0F50E00263E
:100E5200000E012200C0E9FF01C0EAFFC651EE24E4
:100E6200006EC751EE20016ECBCDE1FFCCCDE2FF8B
:100E720000C0E6FF01C0E6FF040E006E000E016E28
:100E8200CACD04F0000E056E4FEC02F0F50E0026FE
:100E9200000E0122020E0024CB6F000E0120CC6F47
:100EA200040E006E000E016ECACD04F0000E056E37
:100EB2004FEC02F0F50E0026000E0122020E002475
:100EC200E96E000E0120EA6EC651EE5C006EC7515B
:100ED200EE58016ECBCDE1FFCCCDE2FF00C0E6FFC4
:100EE20001C0E6FF2CD0040E006E000E016ECACDCA
:100EF20004F0000E056E4FEC02F0F50E0026000E17
:100F0200012200C0E1FF01C0E2FFE66AE66A040EC8
:100F1200006E000E016ECACD04F0000E056E4FEC9D
:100F220002F0F50E0026000E0122020E0024E16EF0
:100F3200000E0120E26EE66AE66A0001E307C8CD10
:100F420000F0C9CD01F007D00D01CA2BE6D6C8CDFD
:080F520000F0C9CD01F012000E
:100F5A000D01C66BC76B130EC75DD8B06AD1C653F5
:100F6A00D8A467D1C751010FC86F800E006E800EDA
:100F7A00000A005C02E1140EC85DD8B058D1C6530D
:100F8A00D8A455D1040E006E000E016EC7CD04F030
:100F9A00000E056E4FEC02F0F50E0026000E01223F
:100FAA0000C0E9FF01C0EAFFEECFD6FDEECFD7FDC4
:100FBA00040E006E000E016EC7CD04F0000E056E21
:100FCA004FEC02F0F50E0026000E0122020E00245C
:100FDA00E96E000E0120EA6EEECFD8FDEECFD9FD04
:100FEA00040E006E000E016EC8CD04F0000E056EF0
:100FFA004FEC02F0F50E0026000E012200C0E9FFB8
:10100A0001C0EAFFEECFDAFDEECFDBFD040E006E83
:10101A00000E016EC8CD04F0000E056E4FEC02F012
:10102A00F50E0026000E0122020E0024E96E000EC3
:10103A000120EA6EEECFDCFDEECFDDFD17EC02F00B
:10104A0000C0C9FDC951010A77E1040E006E000E05
:10105A00016EC7CD04F0000E056E4FEC02F0F50EDE
:10106A000026000E0122020E0024CA6F000E012083
:10107A00CB6F040E006E000E016EC7CD04F0000E99
:10108A00056E4FEC02F0F50E0026000E0122020E4C
:10109A000024E96E000E0120EA6E040E006E000EB6
:1010AA00016EC8CD04F0000E056E4FEC02F0F50E8D
:1010BA000026000E0122020E0024D96E000E012025
:1010CA00DA6EDE50EE24006EDE50EE20016ECACDDE
:1010DA00E1FFCBCDE2FF00C0E6FF01C0E6FF040E50
:1010EA00006E000E016EC8CD04F0000E056E4FECC6
:1010FA0002F0F50E0026000E012200C0E1FF01C039
:10110A00E2FFE66AE66A040E006E000E016EC8CDC2
:10111A0004F0000E056E4FEC02F0F50E0026000EEC
:10112A000122020E0024E16E000E0120E26EE66A40
:10113A00E66A010EC66F79D0C951020A76E1040E39
:10114A00006E000E016EC8CD04F0000E056E4FEC65
:10115A0002F0F50E0026000E0122020E0024CA6FCC
:10116A00000E0120CB6F040E006E000E016EC8CD7A
:10117A0004F0000E056E4FEC02F0F50E0026000E8C
:10118A000122020E0024E96E000E0120EA6E040E0E
:10119A00006E000E016EC7CD04F0000E056E4FEC16
:1011AA0002F0F50E0026000E0122020E0024D96E6E
:1011BA00000E0120DA6EDE50EE24006EDE50EE20C4
:1011CA00016ECACDE1FFCBCDE2FF00C0E6FF01C050
:1011DA00E6FF040E006E000E016EC7CD04F0000E8D
:1011EA00056E4FEC02F0F50E0026000E012200C03B
:1011FA00E1FF01C0E2FFE66AE66A040E006E000E35
:10120A00016EC7CD04F0000E056E4FEC02F0F50E2C
:10121A000026000E0122020E0024E16E000E0120BB
:10122A00E26EE66AE66A010EC66FC82B9ED6C72B27
:10123A0092D6C651010AD8B48BD60001E36B0D01D0
:10124A00C76B800E006E800E000A005C02E1140E6D
:10125A00C75D23E2040E006E000E016EC7CD04F0D6
:10126A00000E056E4FEC02F0F50E0026000E01226C
:10127A0000C0E9FF01C0EAFFEECF01F0EECF02F0B5
:10128A00000E006E0250005C02E10150000802E20A
:10129A000001E32B0D01C72BD4D701014D6B1200BE
:1012AA00060E0C6E2B0E0D6E0D2EFED70C2EFCD7D5
:0212BA00120020
:0C12BC00020E0D6E0D2EFED70000120079
:0A12C800850E0D6E0D2EFED71200EC
:0E12D200CF0E0D6E0D2EFED700000000120094
:1012E0000D01C651200A09E0C6510D0804E3090E9C
:1012F000C65D01E302D0006A02D0010E006E12004A
:101300000D01C651390806E3300EC65D03E3010E38
:08131000006E01D0006A12001A
:10131800800E0D01C719006E800E005C02E1000E00
:10132800C65D08E2C6510008006EC7CD01F0000E88
:0E133800015604D0C6CD00F0C7CD01F0120062
:101346000450000A08E10550000A05E1FF0E006E90
:101356007F0E016E58D00D6A096A086A01500010A6
:10136600D8B4000C015005180A6E0ABE0D1E0B6A91
:1013760005AE05D0041E051E042AD8B4052A01AE02
:1013860005D0001E011E002AD8B4012A01500510FE
:101396000A6E0ABE10D077EC02F00BB020D00DAE6C
:1013A600000C001E011E002AD8B4012A081E091EC0
:1013B600082AD8B4092A000C05AE0DD001BE07D004
:1013C6000150096E0050086E016A006AE8D7016A8A
:1013D600006A002A000C011E001E0B2ADDD7082A0F
:1013E600D8B4092A0450085CD8A4D9D70550095C9A
:1013F600D8A4D5D7096A086A002AD8B4012A01AE4A
:08140600CED70000FF0C12001C
:10140E00220E0C6E086A096A0A6A0B6A0C06D8B4B8
:10141E001FD0D8900B320A32093208320332023210
:10142E0001320032D8A0F2D70C06D8B409D004503D
:10143E0008260550092206500A2207500B22EAD729
:10144E00045008260550092206500A2207500B2286
:02145E0012007A
:10146000086A096A000E07620364B5EF0AF00250C9
:1014700006180A6E075003267E0ED8A046EF0AF023
:10148000035ED8B0BAEF0AF04AEF0AF0035ED8A0C4
:10149000BFEF0AF0028E068E02C00EF001C00BF004
:1014A00000C00DF000500402F4CF0CF00150050212
:1014B000F4CF00F0F3CF08F00402F3500C26F45000
:1014C0000822000E00220D500502F3500C26F450A5
:1014D0000822000E002202500402F3500826F450A5
:1014E000002202500502016A000E0122F35000267C
:1014F000F45001220D500602F3500826F450002249
:10150000026A000E012202220B500602F35000264E
:10151000F4500122000E02220E500602F350012662
:10152000F450022202BE9DEF0AF008360036013662
:1015300002360306D8B4BFEF0AF0B0EF0AF0D88045
:10154000800E08640030000E002201220222D8A082
:10155000B0EF0AF0023201320032034ABAEF0AF069
:101560000AAE029E000EC2EF0AF0010EB8EC01F0C6
:10157000C2EF0AF0020EBFEC01F0C2EF0AF0040E57
:06158000ABEC01F01200CB
:101586000A6A0350D8A40A800750D8A40A820A50CF
:10159600D8B426EF0BF0030AD8B4DFEF0AF00AB08E
:1015A600DAEF0AF006AE24EF0BF022EF0BF002AEF4
:1015B60022EF0BF024EF0BF00250800B0A6E029E16
:1015C6000650800B069E0A18D8B4F0EF0AF00A50AF
:1015D600D8B422EF0BF024EF0BF00750035CD8B41D
:1015E600FAEF0AF0D8A016EF0BF01CEF0BF006503E
:1015F600025CD8B404EF0BF0D8A016EF0BF01CEF8A
:101606000BF00550015CD8B40EEF0BF0D8A016EF26
:101616000BF01CEF0BF00450005CD8B426EF0BF077
:10162600D8B01CEF0BF00A52D8B424EF0BF022EF1F
:101636000BF00A52D8B422EF0BF024EF0BF0D8804F
:0E1646001200D8901200D880D8841200120032
:101654000050086E0150006E0250016E0350026E7D
:10166400036A0B6A0C6A9E0E036E0A6A02AE47EFA7
:101674000BF0081E001E011E021E082AD8B4002A00
:10168400D8B4012AD8B4022A0A8E020E0C6EA3EC36
:0416940002F012004E
:1016980003500718D8A460EF0BF002500618D8A41E
:1016A80060EF0BF001500518D8A460EF0BF0005064
:0E16B8000418D8B4D8841200D894120012007E
:1016C600C6CD02F0C7CD03F002C000F003C001F0A2
:1016D600024A032A00C0E9FF01C0EAFFEE5201E018
:1016E600F3D70D01C651025C006EC7510358016E57
:0A16F600010E005E000E015A120002
:101700000D01D16BD26BD36BD46BD56B8B946751BE
:101710006C03F3CFD4FDF4CFD5FDD44BD52B695159
:10172000CA5D006E016A000E015AD4CD04F0D5CD19
:1017300005F04FEC02F0050E0024D46F000E0120DE
:10174000D56FD4516525E96ED5516621EA6EEECF8D
:10175000D2FDD44BD52BCE6BCE51D25D68E3CD6B91
:10176000CF6B6C51CF5D61E2CE51D21902E1D16BEA
:1017700008D0D4516525E96ED5516621EA6EEECFC9
:10178000D1FDD44BD52BD1CDD3FDD06B080ED05D80
:101790004AE26851CD5D01E346D0010ED315016EDA
:1017A0000150010A1DE1CE51C625D66F000EC7219A
:1017B000D76F080ECF03F3CF00F0F4CF01F0005045
:1017C000C825D86F0150C921D96FD051D827000E34
:1017D000D923CBCDDAFDCCCDDBFDE1EC01F01DD082
:1017E0000D01CE51C625D66F000EC721D76F080E4A
:1017F000CF03F3CF00F0F4CF01F00050C825D86F2D
:101800000150C921D96FD051D827000ED92335C036
:10181000DAFD36C0DBFDE1EC01F00D01CD2BD33359
:10182000D39FD02BB3D7CF2B9CD7CE2B95D78B84E0
:06183000D2CD00F0120011
:101836000D0E0D01D66FCBEC01F00A0E0D01D66F21
:06184600CBEC01F01200E2
:0C184C003A0E0D6E0D2EFED700001200AB
:10185800B0CDDEFDB1CDDFFDB2CDE0FDB3CDE1FD14
:10186800B4CDE2FDB5CDE3FDB6CDE4FDB7CDE5FDE4
:101878001FEC01F00D01B251B65D006EB351B759BE
:10188800016E010E0024046E000E0120056EB05199
:10189800B45D006EB151B559016E004A012A4FEC92
:1018A80002F000C0BAFD01C0BBFDB9CD00F0016A6D
:1018B80000C0DEFDB8CDDFFD9DEC01F0010E0D018D
:1018C800BA5F000EBB5B000E006EBB51005C02E10C
:0818D800BA510008EAE3120016
:1018E0000D01B251B31108E0B2CDE1FFB3CDE2FF7B
:1018F000B0CDE6FFB1CDE6FFB0CDE9FFB1CDEAFF57
:10190000EECF00F000C0B6FD00C0C6FDE9DC00521D
:1019100003E0B04BB12BF0D7B46B000EB6BFFF0E97
:10192000006E000E001802E12D0EB61905E1010E41
:10193000B46FB04BB12B0CD0000EB6BFFF0E006ED3
:10194000000E001802E12B0EB61902E1B04BB12BCC
:10195000B66BB76BB86BB96BBA6BB56BB4B90BD070
:10196000B0CDE9FFB1CDEAFFEE502E0A04E1B48913
:10197000B04BB12B52D0B0CDE9FFB1CDEAFFEECFE5
:10198000C6FDBEDC005201E149D0B483B651080A5D
:101990003FE0B4A901D0B507B62BB7CD00F0B8CD64
:1019A00001F0B9CD02F0BACD03F00A0E046E000EBC
:1019B000056E066E076E2BDD00C0B7FD01C0B8FDD9
:1019C00002C0B9FD03C0BAFD00000000B0CDE9FFC0
:1019D000B1CDEAFF300EEE5C006E016A000E015AD6
:1019E000000E01BEFF0E026E036EB7510026B85105
:1019F0000122B9510222BA51032200C0B7FD01C031
:101A0000B8FD02C0B9FD03C0BAFD0000000003D05C
:101A1000B4B901D0B52BB04BB12BA0D7B66BB0CDBC
:101A2000E9FFB1CDEAFFEE50650A08E0B0CDE9FF6D
:101A3000B1CDEAFFEE50450A01E065D0B04BB12BC5
:101A4000B0CDE9FFB1CDEAFFEE502D0A04E1B48735
:101A5000B04BB12B09D0B0CDE9FFB1CDEAFFEE50CC
:101A60002B0A02E1B04BB12BB0CDE9FFB1CDEAFFBB
:101A7000EE50300A03E1B04BB12BF6D7B0CDE9FF01
:101A8000B1CDEAFFEECFC6FD3BDC005237E0B0CD72
:101A9000E9FFB1CDEAFF300EEE5CB66FB04BB12B73
:101AA000B0CDE9FFB1CDEAFFEECFC6FD29DC005293
:101AB00025E00A0EB603F3CFB6FDB0CDE9FFB1CDF8
:101AC000EAFF300EEE5C006E0050B627B04BB12B33
:101AD000B0CDE9FFB1CDEAFFEECFC6FD11DC00527B
:101AE0000DE00A0EB603F3CFB6FDB0CDE9FFB1CDE0
:101AF000EAFF300EEE5C006E0050B627B4A703D0AC
:101B0000B6510008B66FB651B527000EB31902E101
:101B1000000EB2190AE0B4A308D0B2CDE1FFB3CDF4
:101B2000E2FFB0CDE6FFB1CDE6FFB7CD00F0B8CD16
:101B300001F0B9CD02F0BACD03F08CDD00C0B7FDE5
:101B400001C0B8FD02C0B9FD03C0BAFD046A056A50
:101B5000066A076AB7CD00F0B8CD01F0B9CD02F042
:101B6000BACD03F099DD010ED8A4000E006E00522C
:101B700005E0006A016A026A036A00D1800EB519A5
:101B8000006E800E000A005CD8B070D0B55100081D
:101B9000B56F800EB519006E800E0A0A005C1CE35A
:101BA000B7CD00F0B8CD01F0B9CD02F0BACD03F059
:101BB000FF0E046EE60E056E5B0E066E5D0E076E82
:101BC0004FDC00C0B7FD01C0B8FD02C0B9FD03C0C5
:101BD000BAFD0A0EB55FDDD7B551000A1BE0B7CDDF
:101BE00000F0B8CD01F0B9CD02F0BACD03F0CD0EC2
:101BF000046ECC0E056E4C0E066E7B0E076E30DC4E
:101C000000C0B7FD01C0B8FD02C0B9FD03C0BAFDF8
:101C1000B507E2D7010E046E000E056E000E066ECB
:101C2000010E076EB7CD00F0B8CD01F0B9CD02F0CE
:101C3000BACD03F0A8DC010ED8B0000E006E005241
:101C400014E0B4A109D0010E006E000E016E800EEA
:101C5000026E030E036E92D0010E006E000E016E36
:101C6000000E026E010E036E89D071D0800E000A44
:101C7000006E800EB519005C6AE20A0EB55D1DE3C8
:101C8000B7CD00F0B8CD01F0B9CD02F0BACD03F078
:101C9000F90E046E020E056E150E066EA00E076E8E
:101CA00030EC0AF000C0B7FD01C0B8FD02C0B9FDBC
:101CB00003C0BAFD0A0EB55FE0D7B551000A1CE0BB
:101CC000B7CD00F0B8CD01F0B9CD02F0BACD03F038
:101CD000000E046E000E056E200E066E820E076E5C
:101CE00030EC0AF000C0B7FD01C0B8FD02C0B9FD7C
:101CF00003C0BAFDB507E1D7B7CD04F0B8CD05F004
:101D0000B9CD06F0BACD07F0FF0E006EFF0E016EE2
:101D10007F0E026EFF0E036E36DC010ED8B0000E91
:101D2000006E005214E0B4A109D0FF0E006EFF0E49
:101D3000016EFF0E026EFF0E036E20D0FF0E006ECE
:101D4000FF0E016E7F0E026EFF0E036E17D0B4A160
:101D50000DD0000EB719006E000EB819016E800E7E
:101D6000B919026E000EBA19036E08D0B7CD00F093
:0E1D7000B8CD01F0B9CD02F0BACD03F01200EB
:101D7E00B2CDF6FFB3CDF7FFB4CDF8FF0900F5CF26
:101D8E0000F0005218E0B2CDF6FFB3CDF7FFB4CDA0
:101D9E00F8FF0900F5CF00F0B0CDE1FFB1CDE2FFC5
:101DAE0000C0E6FF0D01B04BB12B010EB227000EA5
:101DBE00B323B423DDD7B0CDE1FFB1CDE2FFE66AA8
:021DCE00120001
:101DD0000450000A12E10550000A0FE10650000A03
:101DE0000CE10750000A09E1FF0E006EFF0E016EC4
:101DF0007F0E026EFF0E036EA8D0086A096A0750B4
:101E0000D8B493EF0FF00350D8B498EF0FF002500E
:101E100006180A6E028E068E0E6A02C008F001C015
:101E20000CF000C00DF004500D5E0550D8A0053C2C
:101E30000C5E0650D8A0063C085E086A0C6A0D6A63
:101E4000D8A02AEF0FF0D8900232013200320832C7
:101E5000010E0E6E0750035ED8A037EF0FF07E0E16
:101E60000E240326D8B09DEF0FF03DEF0FF07E0E4D
:101E70000E240326D8A0A2EF0FF0180E0B6E0D361D
:101E80000C3608360036013602360E360450005E37
:101E90000550D8A0053C015E0650D8A0063C025E65
:101EA00006340E120EA058EF0FF00D8063EF0FF006
:101EB000045000260550D8B0053C01260650D8B085
:101EC000062802260D900B2E3FEF0FF089EF0FF042
:101ED000D8900036013602360E360450005E0550AA
:101EE000D8A0053C015E0650D8A0063C025E063430
:101EF0000E10010B0D26D8B00C2AD8B4082AD8A48D
:101F000089EF0FF008320C320D32032AD8B49DEF5E
:101F10000FF00AAE089E0850026E0C50016E0D5074
:101F2000006EA5EF0FF0010EC1EC05F0A5EF0FF06C
:101F3000020EB8EC01F0A5EF0FF0040EBFEC01F0BB
:0C1F4000A5EF0FF0080EABEC01F0120052
:101F4C0000C008F00150006E016A026A036A0B6A55
:101F5C000C6A016A026A036A960E036E0A6A00AE84
:101F6C00BEEF0FF0081E001E082AD8B4002A0A8EF5
:101F7C0000C001F008C000F0086A026A2AEC06F002
:021F8C00120041
:101F8E00B2CD01F0010E006E015004E0003600905B
:101F9E00FF0FFBD700C0B6FD001C0D01B56FB46B73
:101FAE00B0CDE9FFB1CDEAFFB36BB351070824E31F
:101FBE00B551EF16120EE926B551EF165EEC09F08B
:101FCE00B651EF125EEC09F0120EE95EB651EF1447
:101FDE00006E0CE0B3CD01F0010E006E015004E076
:101FEE0000360090FF0FFBD70050B41364EC09F0DD
:0E1FFE0064EC09F0B32BD9D7B4CD00F012007B
:08200C00067EB1EC03F01200A6
:102014000B6A0350D8B450EF10F002500A6E028ECF
:102024008E0E035E03AE54EF10F0036C080E035CD7
:10203400D8A02FEF10F0036E013602C001F0026A3F
:10204400080E035CD8A02FEF10F0036E0136016A6E
:102054000350D8A4D89039EF10F00350D8B439EF16
:1020640010F0D89002320132032E33EF10F00BBC83
:1020740001A046EF10F0D8A046EF10F0012AD8B422
:10208400022A02BE63EF10F00AAE69EF10F0021EDE
:10209400011E012AD8B4022A69EF10F0026A016A0B
:1020A40069EF10F00B800BAE6DEF10F0026A0AAE10
:1020B4006DEF10F0FF0E026E016E0A3602326DEF04
:1020C40010F0010E0C6EE0EC05F06FEF10F0000E56
:1020D4000C6E6FEF10F0FF0E0C6E0150006E02508C
:0420E400016E120077
:1020E800B0CD65FDB1CD66FDB0CDE9FFB1CDEAFF5C
:1020F800EECF67FD010E0D01B025E96E000EB1218E
:10210800EA6EEECF68FD020EB025E96E000EB12131
:10211800EA6EEECF69FD030EB025E96E000EB1211F
:10212800EA6EEECF6AFD040EB025E96E000EB1210D
:10213800EA6EEECF6BFD68CD00F00032009E0032F3
:10214800009E0032009E00C06CFD080E046E68CD33
:1021580000F0D2EC01F008C000F0005205E06C512C
:0A216800010F006E00C06CFD1200B4
:102172006B0E0D01C66FAB0EC76F000EC86F94ECED
:1021820003F067CDC6FD580E0D01C76F010EC86F73
:10219200EEEC05F0580EC66F010EC76FC5EC05F0E8
:1021A200E70EC66FA90EC76F000EC86F94EC03F05E
:1021B20068CDC6FD580E0D01C76F010EC86FEEEC5B
:1021C20005F0580EC66F010EC76FC5EC05F0D60EAE
:1021D200C66FA90EC76F000EC86F94EC03F06CCDEA
:1021E200C6FD580E0D01C76F010EC86FEEEC05F06B
:1021F200580EC66F010EC76FC5EC05F0080EC66F0C
:10220200AB0EC76F000EC86F94EC03F06BCDC6FD2A
:10221200580E0D01C76F010EC86FEEEC05F0580E97
:10222200C66F010EC76FC5EC05F01BEC0CF0120077
:10223200B0CDB8FDB1CDB9FDB4CDC6FDB5CDC7FDAC
:1022420063EC0BF000C0BDFD01C0BEFD000EBE5D23
:1022520002E16B51BD5D04E36BCDBDFD000EBE6FAF
:10226200BB6BBC6BBE51BC5D02E1BD51BB5D21E2EB
:10227200B8CDC6FDB9CDC7FDB2CDC8FDB3CDC9FD40
:10228200BB51B425E96EBC51B521EA6EEECFCAFD51
:10229200B6CDCBFDB7CDCCFD80EC0BF000C0BAFDC6
:1022A200BA51B827000EB923B84BB92BBB4BBC2B84
:0422B200D9D7120066
:1022B6000B6A0A6A096A086A0E6A03340836045009
:1022C600085E0550D8A0053C095E0650D8A0063C1D
:1022D6000A5E0750D8A0073C0B5EE86AD8A0010E3C
:1022E6000E5E0336070E0C6E0334083609360A36C0
:1022F6000B360E36045003A012D0085E0550D8A047
:10230600053C095E0650D8A0063C0A5E0750D8A0D8
:10231600073C0B5EE86AD8A0010E0E5E11D00826B7
:102326000550D8B0053C09260650D8B0063C0A260A
:102336000750D8B0073C0B26E86AD8B0010E0E2627
:1023460003360C2ED1D70234083609360A360B3638
:102356000E36045003A012D0085E0550D8A0053CE6
:10236600095E0650D8A0063C0A5E0750D8A0073C76
:102376000B5EE86AD8A0010E0E5E11D00826055045
:10238600D8B0053C09260650D8B0063C0A260750A8
:10239600D8B0073C0B26E86AD8B0010E0E260236E6
:1023A600070E0C6E0234083609360A360B360E3620
:1023B600045002A012D0085E0550D8A0053C095E64
:1023C6000650D8A0063C0A5E0750D8A0073C0B5E14
:1023D600E86AD8A0010E0E5E11D008260550D8B0C6
:1023E600053C09260650D8B0063C0A260750D8B048
:1023F600073C0B26E86AD8B0010E0E2602360C2ED4
:10240600D1D70134083609360A360B360E36045053
:1024160002A012D0085E0550D8A0053C095E065001
:10242600D8A0063C0A5E0750D8A0073C0B5EE86AB7
:10243600D8A0010E0E5E11D008260550D8B0053C76
:1024460009260650D8B0063C0A260750D8B0073CE5
:102456000B26E86AD8B0010E0E260136070E0C6E62
:102466000134083609360A360B360E36045001A0FA
:1024760012D0085E0550D8A0053C095E0650D8A0CB
:10248600063C0A5E0750D8A0073C0B5EE86AD8A057
:10249600010E0E5E11D008260550D8B0053C09265F
:1024A6000650D8B0063C0A260750D8B0073C0B2683
:1024B600E86AD8B0010E0E2601360C2ED1D70034AC
:1024C600083609360A360B360E36045001A012D0ED
:1024D600085E0550D8A0053C095E0650D8A0063C0B
:1024E6000A5E0750D8A0073C0B5EE86AD8A0010E2A
:1024F6000E5E11D008260550D8B0053C09260650B8
:10250600D8B0063C0A260750D8B0073C0B26E86A26
:10251600D8B0010E0E260036070E0C6E00340836B3
:1025260009360A360B360E36045000A012D0085E65
:102536000550D8A0053C095E0650D8A0063C0A5EA8
:102546000750D8A0073C0B5EE86AD8A0010E0E5EC5
:1025560011D008260550D8B0053C09260650D8B03B
:10256600063C0A260750D8B0073C0B26E86AD8B0C6
:10257600010E0E2600360C2ED1D700B00ED0045018
:1025860008260550D8B0053C09260650D8B0063CAA
:0C2596000A260750D8B0073C0B261200A4
:1025A2000001E45308E10D01B151000A02E1000EFD
:1025B200B01901E001D06CD10D01B66BB46B800E85
:1025C200006E800E000A005C02E1140EB45DD8B009
:1025D200EED0B0CDD6FDB1CDD7FDB2CDD8FDB3CDC5
:1025E200D9FD040E006E000E016EB4CD04F0000E93
:1025F200056E4FEC02F0F50E0026000E012200C01F
:10260200E9FF01C0EAFFEECFDAFDEECFDBFD040EFB
:10261200006E000E016EB4CD04F0000E056E4FEC9C
:1026220002F0F50E0026000E0122020E0024E96ED1
:10263200000E0120EA6EEECFDCFDEECFDDFD17ECE1
:1026420002F000C0B5FDB551010A6EE1040E006E44
:10265200000E016EB4CD04F0000E056E4FEC02F0D8
:10266200F50E0026000E012200C0B7FD01C0B8FD24
:10267200040E006E000E016EB4CD04F0000E056E65
:102682004FEC02F0F50E0026000E012200C0E9FF19
:1026920001C0EAFFB251EE5C006EB351EE58016E1A
:1026A200B7CDE1FFB8CDE2FF00C0E6FF01C0E6FF13
:1026B200040E006E000E016EB4CD04F0000E056E25
:1026C2004FEC02F0F50E0026000E0122020E00244D
:1026D200B76F000E0120B86F040E006E000E016E7F
:1026E200B4CD04F0000E056E4FEC02F0F50E00269C
:1026F200000E0122020E0024E96E000E0120EA6E95
:10270200B251EE24006EB351EE20016EB7CDE1FF5F
:10271200B8CDE2FF00C0E6FF01C0E6FF010EB66FD2
:10272200010E01014D6F43D00D01B551020A3CE18A
:10273200040E006E000E016EB4CD04F0000E056EA4
:102742004FEC02F0F50E0026000E0122020E0024CC
:10275200B76F000E0120B86F040E006E000E016EFE
:10276200B4CD04F0000E056E4FEC02F0F50E00261B
:10277200000E0122020E0024E96E000E0120EA6E14
:10278200B251EE24006EB351EE20016EB7CDE1FFDF
:10279200B8CDE2FF00C0E6FF01C0E6FF010EB66F52
:1027A200010E01014D6F03D00D01B42B08D70D01AD
:1027B200B65365E1B46B800E006E800E000A005CB9
:1027C20002E1140EB45D50E2040E006E000E016EC2
:1027D200B4CD04F0000E056E4FEC02F0F50E0026AB
:1027E200000E012200C0E9FF01C0EAFFEECF01F0B6
:1027F200EECF02F00250000A02E1000E011831E1B0
:10280200040E006E000E016EB4CD04F0000E056ED3
:102812004FEC02F0F50E0026000E012200C0E1FF8F
:1028220001C0E2FFB0CDE6FFB1CDE6FF040E006EBF
:10283200000E016EB4CD04F0000E056E4FEC02F0F6
:10284200F50E0026000E0122020E0024E16E000E9B
:102852000120E26EB2CDE6FFB3CDE6FF0001E32B2D
:1028620003D00D01B42BA7D7000E000A03E10D011E
:10287200140EB41904E1010E0001E46F09D0000145
:10288200E351130A02E1ADEC07F00D01B06BB16B3D
:02289200120032
:10289400290E0B6E960E0C6E7F0E0D6E0D2EFED74E
:0A28A4000C2EFCD70B2EFAD7120001
:1028AE000D01B46B050EB45D0AE2B451B225E16EB2
:1028BE00000EB321E26E200EE66EB42BF3D7B451A8
:1028CE00B225E16E000EB321E26EE66AB407B45192
:1028DE00B225B56F000EB321B66F0A0E046E000E50
:1028EE00056EB0CD00F0B1CD01F066EC06F008C07B
:1028FE0000F009C001F0300E0026B5CDE1FFB6CDD7
:10290E00E2FF00C0E6FF0A0E046E000E056EB0CDAB
:10291E0000F0B1CD01F066EC06F000C0B0FD01C0D4
:10292E00B1FD000E011802E1000E001801E102D007
:06293E00B407CDD7120022
:0A294400B0CD35F0B1CD36F0120031
:10294E00B2CD01F0010E006E015004E00036009091
:10295E00FF0FFBD700C0B4FD001EB0CDE9FFB1CD17
:10296E00EAFF0050EF16120EE9260050EF1655EC56
:10297E0009F00D01B451EF12120EE95E69EC09F087
:10298E00B451EF14B36FB351000A000ED8A4010E68
:0C299E00B36F55EC09F0B3CD00F012004F
:1029AA00B0CDC6FDB1CDC7FD81EC06F000C0B2FDC9
:1029BA0001C0B3FD0D01B351000A02E1000EB219C4
:1029CA000FE101014D530CE0ADEC07F0B0CDC6FDAF
:1029DA00B1CDC7FD81EC06F000C0B2FD01C0B3FD68
:0A29EA00B2CD00F0B3CD01F01200F1
:1029F400B2CD01F0010E006E015004E000360090EB
:102A0400FF0FFBD700C0B6FD001E00C0B5FDB0CD62
:102A1400E9FFB1CDEAFF0050EF16120EE9260D01D1
:102A2400B46BB451070816E3B4CD00F0B3CD01F094
:102A3400005004E00132019EFF0FFBD7B551EF16A1
:102A440001A002D0B651EF1269EC09F0B651EF12B1
:102A5400B42BE7D7120EE95E64EC09F064EC09F0DC
:022A640012005E
:102A66000D01B251B65DC66FB351B759C76F8CEC45
:102A760009F000C0C4FD01C0C5FDB051B45DC66F0C
:102A8600B151B559C76F8CEC09F0800E0118BA6FB9
:102A9600800EC519BA5D02E1C451005C010ED8B0C2
:102AA600000EBA6F000EBB6F8B94BA51BB1114E0C7
:102AB600B0CDEAFDB1CDEBFDB2CDECFDB3CDEDFD74
:102AC6008CEC00F0B4CDEAFDB5CDEBFDB6CDECFD5A
:102AD600B7CDEDFD8CEC00F0800EB519006E800EC2
:102AE600B119005C02E1B051B45D14E2B0CDEAFD6B
:102AF600B1CDEBFDB4CDECFDB5CDEDFD8CEC00F02C
:102B0600B2CDEAFDB3CDEBFDB6CDECFDB7CDEDFD17
:102B16008CEC00F0B051B45DBC6FB151B559BD6FCE
:102B2600B251B65DC66FB351B759C76F8CEC09F099
:102B360000C0BEFD01C0BFFD020E046E000E056E94
:102B4600BCCD00F0BDCD01F0A3EC09F000C0C0FD86
:102B560001C0C1FD800E0D01B319006E800EB719BC
:102B6600005C02E1B651B25D05E2010EC26F000ED5
:102B7600C36F04D0FF0EC26FFF0EC36F800EB51970
:102B8600006E800EB119005C02E1B051B45D39E30C
:102B9600BA51BB110FE0B2CDD6FDB3CDD7FDB0CD46
:102BA600D8FDB1CDD9FDB8CDDAFDB9CDDBFDE1EC6F
:102BB60001F00ED0B0CDD6FDB1CDD7FDB2CDD8FD4A
:102BC600B3CDD9FDB8CDDAFDB9CDDBFDE1EC01F031
:102BD6000D01BE51C05FBF51C15B800EC119006EB1
:102BE600800E005C02E1000EC05D08E2C251B22711
:102BF600C351B323BC51C027BD51C123B04BB12B28
:062C0600BDD78B84120013
:102C0C00040E046EB0CD00F0D2EC01F008C000F060
:102C1C0000C0B0FD25D0B00E336E000E346EDC0E4D
:102C2C000D01976F000E986F28D0DC0E336E000EDE
:102C3C00346EB00E976F000E986F1FD0B00E336EBF
:102C4C00000E346EDC0E976F000E986F16D0DC0EF3
:102C5C00336E000E346EB00E976F000E986F0DD061
:102C6C000D01B051000AD7E0B051010ADEE0B051BD
:0C2C7C00020AE4E0B051030AEAE0120092
:062C8800B0CD2EF0120099
:102C8E0099CDF1F09ACDF2F09BCDF3F09CCDF4F00E
:102C9E009DCDEDF09ECDEEF09FCDEFF0A0CDF0F0FE
:102CAE00A1CDE5F0A2CDE6F0A3CDE7F0A4CDE8F0FE
:102CBE00A5CDE9F0A6CDEAF0A7CDEBF0A8CDECF0CE
:022CCE001200F2
:102CD000C26A1B1C006E0050C1160F0EC012C08EBF
:102CE00099CD00F000360090003600900050C212DE
:102CF000C28026EC0CF0C282C2A201D0FDD7C4CFA4
:102D000001F0006A00C09AFD01C09BFDC350001293
:102D1000000E011200C09AFD01C09BFDC290000E82
:102D20000014026E0150800B036E000E031802E1C6
:102D3000000E021803E00D019A6B9B6B9ACD00F018
:062D40009BCD01F0120022
:102D4600960E0001ED6F030EEE6FD60EEF6F0D0EB1
:102D5600F06FFF0EF16FFF0EF26F000EF36F000EB5
:102D6600F46FFF0EE56FFF0EE66F000EE76F000EC5
:102D7600E86FFF0EE96FFF0EEA6F000EEB6F000EB5
:102D8600EC6FAC8A900EAB6E948E949C9EAA03D088
:082D9600AECF00F0FBD71200E4
:102D9E000900F5CFE6FF0006FBE10106F9E112009E
:102DAE000D019F51000805E3070EA06F000EA16FE5
:102DBE0012D09F51160805E2170EA26F000EA36FD8
:102DCE0006D09F51010FA26FA36B000EA323A2CDBD
:102DDE00A0FDA3CDA1FDA0CDAAFDA1CDABFDA46B01
:102DEE00A56B046A056A066A076A99CD00F09ACD4A
:102DFE0001F09BCD02F09CCD03F0C3EC0AF0010E66
:102E0E00D8B0000E006E005209E09DCDE1FF9ECDC0
:102E1E00E2FF2D0EE66E9D4B9E2B9B7F99CD04F00F
:102E2E009ACD05F09BCD06F09CCD07F0006A016AA5
:102E3E00026A036AC3EC0AF0010ED8B0000E006EEF
:102E4E00005237E0000E046E000E056E000E066E88
:102E5E007F0E076E99CD00F09ACD01F09BCD02F05A
:102E6E009CCD03F0C3EC0AF0010ED8B0000E006E3C
:102E7E0000521FE099CD00F09ACD01F09BCD02F0EB
:102E8E009CCD03F0000E046E000E056E200E066E35
:102E9E00820E076E30EC0AF000C099FD01C09AFD5B
:102EAE0002C09BFD03C09CFD010EA45F000EA55B3E
:102EBE00C9D7000E046E000E056E200E066E820E31
:102ECE00076E99CD00F09ACD01F09BCD02F09CCD0E
:102EDE0003F0C3EC0AF0000ED8B0010E006E0052E3
:102EEE001EE0000E046E000E056E200E066E820EA3
:102EFE00076E99CD00F09ACD01F09BCD02F09CCDDE
:102F0E0003F0E8EC0EF000C099FD01C09AFD02C07E
:102F1E009BFD03C09CFD0D01A44BA52BCAD7A4514C
:102F2E00AA27A551AB23010EA66F000EA76FA6CD43
:102F3E0000F0A7CD01F0A6EC0FF000C0ACFD01C073
:102F4E00ADFD02C0AEFD03C0AFFD800EA719006E31
:102F5E00800EAB19005C02E1AA51A65D1EE2000EC6
:102F6E00046E000E056E200E066E820E076EACCD40
:102F7E0000F0ADCD01F0AECD02F0AFCD03F0E8EC38
:102F8E000EF000C0ACFD01C0ADFD02C0AEFD03C031
:102F9E00AFFD0D01A64BA72BD8D7000E046E000E69
:102FAE00056E000E066E800E076EACCD00F0ADCD38
:102FBE0001F0AECD02F0AFCD03F0E8EC0EF099CDFE
:102FCE0004F09ACD05F09BCD06F09CCD07F0B1EC48
:102FDE0003F000C099FD01C09AFD02C09BFD03C025
:102FEE009CFD000E046E000E056E200E066E820E07
:102FFE00076E99CD00F09ACD01F09BCD02F09CCDDD
:10300E0003F0C3EC0AF0000ED8B0010E006E0052B1
:10301E000BE0000E0D01996F000E9A6F000E9B6F64
:10302E007F0E9C6FA44BA52B0D01800EA519006E73
:10303E00800E005C02E1000EA45D38E29DCDE1FF42
:10304E009ECDE2FF300EE66E9D4B9E2B9DCDE1FF99
:10305E009ECDE2FF2E0EE66E9D4B9E2B800EAB1983
:10306E00006E800E005C02E1000EAA5D04E2AA5121
:10307E00A45FAB51A55BFF0EA66FFF0EA76F800E70
:10308E00A519006E800EA719005C02E1A651A45D81
:10309E000DE29DCDE1FF9ECDE2FF300EE66E9D4B23
:1030AE009E2B010EA65F000EA75BE9D7A66BA76B42
:1030BE00800EA719006E800EAB19005C02E1AA51BA
:1030CE00A65D6CE299CD00F09ACD01F09BCD02F099
:1030DE009CCD03F00AEC10F000C0A8FD01C0A9FDC4
:1030EE00300EA825006E9DCDE1FF9ECDE2FF00C003
:1030FE00E6FF9D4B9E2BA751A51902E1A451A619DF
:10310E0008E19DCDE1FF9ECDE2FF2E0EE66E9D4BBA
:10311E009E2BA8CD00F0A9CD01F0A6EC0FF000C0BB
:10312E00ACFD01C0ADFD02C0AEFD03C0AFFDACCD28
:10313E0004F0ADCD05F0AECD06F0AFCD07F099CDD4
:10314E0000F09ACD01F09BCD02F09CCD03F006EC81
:10315E0010F000C099FD01C09AFD02C09BFD03C096
:10316E009CFD99CD00F09ACD01F09BCD02F09CCD47
:10317E0003F0000E046E000E056E200E066E820E1B
:10318E00076E30EC0AF000C099FD01C09AFD02C036
:10319E009BFD03C09CFDA64BA72B8AD79DCDE1FFBF
:0831AE009ECDE2FFE66A12006B
:1031B600FF0E01014F6FFF0E506FFF0E516FFF0E96
:1031C600526FC26A1B1C006E0050C1160F0EC01251
:0631D600C08EC280120051
:1031DC000D019B6B9C6B2F6A306A316A326A800ED0
:1031EC00B06F0F0EB16F030EB26FA7EC14F0800E20
:1031FC00B06F0F0EB16F030EB26FCC0EB36FFAEC53
:10320C0014F0800EB06F0F0EB16F030EB26F440E40
:10321C00B36FFAEC14F0020E0C6E730E0D6E0D2ED5
:10322C00FED70C2EFCD7800EB06F0F0EB16F030EB5
:10323C00B26FA7EC14F0800EB06F0F0EB16F030ECF
:10324C00B26FCC0EB36FFAEC14F0800EB06F0F0EA1
:10325C00B16F030EB26FBE0EB36FFAEC14F0800EAA
:10326C00B06F0F0EB16F030EB26FC7EC0FF000C052
:10327C0099FD800EB06F0F0EB16F030EB26FC7ECDD
:10328C000FF000C09AFD9ACD9BFD000E9C6F9BCD5C
:10329C009CFD9B6B99519B13000E9C130F0E9B1561
:1032AC00006E9CCD01F0000E0116A6EC0FF0000E86
:1032BC00046E000E056E000E066E7B0E076E30EC73
:1032CC000AF000C02FF001C030F002C031F003C092
:1032DC0032F0040E026E9BCD00F09CCD01F002503A
:1032EC0007E001320032019E01BC018EFF0FF8D7BE
:1032FC00A6EC0FF02FC004F030C005F031C006F082
:10330C0032C007F0B1EC03F000C02FF001C030F078
:0A331C0002C031F003C032F01200CD
:10332600170E0D01C66FAB0EC76F000EC86F94EC7B
:1033360003F084D3DB0E0D01C66FAA0EC76F000E15
:10334600C86F94EC03F0A50E0D016D6F020E6E6F43
:103356006DCDB0FD6ECDB1FD580EB26F010EB36FDF
:1033660057EC14F0580EC66F010EC76FC5EC05F08A
:103376001BEC0CF06DCDB0FD6ECDB1FDD5EC14F0AF
:1033860000C053F101C054F10101556B566B0D019C
:103396006E510101565D04E10D016D510101555D4E
:1033A6001AE255515325E16E56515421E26E160E1E
:1033B6005525F66EA10E5621F76E000EF86E000E1C
:1033C60056BFFF0EF8220900F5CF00F000C0E6FF59
:1033D600554B562BDCD753C1B0FD54C1B1FD74EC2F
:1033E60010F0B9EC10F071D32B0E0D01C66FAA0EBA
:1033F600C76F000EC86F94EC03F0650E0D016D6F7C
:10340600090E6E6F6DCDB0FD6ECDB1FD580EB26F6B
:10341600010EB36F57EC14F0580EC66F010EC76F4E
:10342600C5EC05F01BEC0CF06DCDB0FD6ECDB1FD1D
:10343600D5EC14F000C053F101C054F10101556BF5
:10344600566B0D016E510101565D04E10D016D5182
:103456000101555D1AE255515325E16E565154212D
:10346600E26E7D0E5525F66E680E5621F76E000E3D
:10347600F86E000E56BFFF0EF8220900F5CF00F0D9
:1034860000C0E6FF554B562BDCD753C1B0FD54C1E7
:10349600B1FD74EC10F0B9EC10F017D3E80E0D0185
:1034A600C66FA80EC76F000EC86F94EC03F0150E1A
:1034B6000D016D6F040E6E6F6DCDB0FD6ECDB1FD5D
:1034C600580EB26F010EB36F57EC14F0580EC66F5C
:1034D600010EC76FC5EC05F01BEC0CF06DCDB0FD11
:1034E6006ECDB1FDD5EC14F000C053F101C054F11E
:1034F6000101556B566B0D016E510101565D04E1DC
:103506000D016D510101555D1AE255515325E16ECC
:1035160056515421E26E010E5525F66E9D0E56212A
:10352600F76E000EF86E000E56BFFF0EF822090069
:10353600F5CF00F000C0E6FF554B562BDCD753C144
:10354600B0FD54C1B1FD74EC10F0B9EC10F0BDD271
:10355600F90E0D01C66FAA0EC76F000EC86F94EC68
:1035660003F0250E0D016D6F040E6E6F6DCDB0FD6F
:103576006ECDB1FD580EB26F010EB36F57EC14F05D
:10358600580EC66F010EC76FC5EC05F01BEC0CF0AC
:103596006DCDB0FD6ECDB1FDD5EC14F000C053F18C
:1035A60001C054F10101556B566B0D016E510101BD
:1035B600565D04E10D016D510101555D1AE255514B
:1035C6005325E16E56515421E26EDC0E5525F66EFA
:1035D600980E5621F76E000EF86E000E56BFFF0EBF
:1035E600F8220900F5CF00F000C0E6FF554B562B38
:1035F600DCD753C1B0FD54C1B1FD74EC10F0B9EC89
:1036060010F063D2FC0E0D01C66FA80EC76F000E38
:10361600C86F94EC03F0FF0E0D016D6F040E6E6F14
:103626006DCDB0FD6ECDB1FD580EB26F010EB36F0C
:1036360057EC14F0580EC66F010EC76FC5EC05F0B7
:103646001BEC0CF06DCDB0FD6ECDB1FDD5EC14F0DC
:1036560000C053F101C054F10101556B566B0D01C9
:103666006E510101565D04E10D016D510101555D7B
:103676001AE255515325E16E56515421E26EDD0E84
:103686005525F66E930E5621F76E000EF86E000E57
:1036960056BFFF0EF8220900F5CF00F000C0E6FF86
:1036A600554B562BDCD753C1B0FD54C1B1FD74EC5C
:1036B60010F0B9EC10F009D2AA0E0D01C66FA80ED3
:1036C600C76F000EC86F94EC03F00F0E0D016D6FFF
:1036D600090E6E6F6DCDB0FD6ECDB1FD580EB26F99
:1036E600010EB36F57EC14F0580EC66F010EC76F7C
:1036F600C5EC05F01BEC0CF06DCDB0FD6ECDB1FD4B
:10370600D5EC14F000C053F101C054F10101556B22
:10371600566B0D016E510101565D04E10D016D51AF
:103726000101555D1AE255515325E16E565154215A
:10373600E26E130E5525F66E7B0E5621F76E000EC1
:10374600F86E000E56BFFF0EF8220900F5CF00F006
:1037560000C0E6FF554B562BDCD753C1B0FD54C114
:10376600B1FD74EC10F0B9EC10F0AFD16E0E0D0196
:10377600C66FAA0EC76F000EC86F94EC03F00F0E4B
:103786000D016D6F090E6E6F6DCDB0FD6ECDB1FD85
:10379600580EB26F010EB36F57EC14F0580EC66F89
:1037A600010EC76FC5EC05F01BEC0CF06DCDB0FD3E
:1037B6006ECDB1FDD5EC14F000C053F101C054F14B
:1037C6000101556B566B0D016E510101565D04E109
:1037D6000D016D510101555D1AE255515325E16EFA
:1037E60056515421E26E220E5525F66E840E562150
:1037F600F76E000EF86E000E56BFFF0EF822090097
:10380600F5CF00F000C0E6FF554B562BDCD753C171
:10381600B0FD54C1B1FD74EC10F0B9EC10F055D107
:10382600250E0D01C66FAB0EC76F000EC86F94EC68
:1038360003F0AC0E0D016D6F060E6E6F6DCDB0FD13
:103846006ECDB1FD580EB26F010EB36F57EC14F08A
:10385600580EC66F010EC76FC5EC05F01BEC0CF0D9
:103866006DCDB0FD6ECDB1FDD5EC14F000C053F1B9
:1038760001C054F10101556B566B0D016E510101EA
:10388600565D04E10D016D510101555D1AE2555178
:103896005325E16E56515421E26E310E5525F66ED2
:1038A6008D0E5621F76E000EF86E000E56BFFF0EF7
:1038B600F8220900F5CF00F000C0E6FF554B562B65
:1038C600DCD753C1B0FD54C1B1FD74EC10F0B9ECB6
:1038D60010F0FBD0560E0D01C66FA70EC76F000E77
:1038E600C86F94EC03F02D0E0D016D6F0A0E6E6F0E
:1038F6006DCDB0FD6ECDB1FD580EB26F010EB36F3A
:1039060057EC14F0580EC66F010EC76FC5EC05F0E4
:103916001BEC0CF06DCDB0FD6ECDB1FDD5EC14F009
:1039260000C053F101C054F10101556B566B0D01F6
:103936006E510101565D04E10D016D510101555DA8
:103946001AE255515325E16E56515421E26E500E3E
:103956005525F66E5E0E5621F76E000EF86E000EB9
:1039660056BFFF0EF8220900F5CF00F000C0E6FFB3
:10397600554B562BDCD753C1B0FD54C1B1FD74EC89
:1039860010F0B9EC10F0A1D0280E0D01C66FA80EEC
:10399600C76F000EC86F94EC03F0310E0D016D6F0A
:1039A600090E6E6F6DCDB0FD6ECDB1FD580EB26FC6
:1039B600010EB36F57EC14F0580EC66F010EC76FA9
:1039C600C5EC05F01BEC0CF06DCDB0FD6ECDB1FD78
:1039D600D5EC14F000C053F101C054F10101556B50
:1039E600566B0D016E510101565D04E10D016D51DD
:1039F6000101555D1AE255515325E16E5651542188
:103A0600E26EE20E5525F66E710E5621F76E000E29
:103A1600F86E000E56BFFF0EF8220900F5CF00F033
:103A260000C0E6FF554B562BDCD753C1B0FD54C141
:103A3600B1FD74EC10F0B9EC10F047D0000E0D019A
:103A46009A1902E1010E9919D8B474D4000E9A1984
:103A560002E1020E9919D8B4C7D4000E9A1902E1F0
:103A6600030E9919D8B41AD5000E9A1902E1040E5C
:103A76009919D8B46DD5000E9A1902E1050E991957
:103A8600D8B4C0D5000E9A1902E1060E9919D8B419
:103A960013D6000E9A1902E1070E9919D8B466D604
:103AA600000E9A1902E1080E9919D8B4B9D6000E7B
:103AB6009A1902E1090E9919D8B40CD7000E9A1971
:0C3AC60002E10A0E9919D8B45FD7120073
:103AD2006F0E0D01B06F0D0EB16F9DCDB2FD9ECD7B
:103AE200B3FD9FCDB4FDBFEC0EF099CDB0FD9ACDE4
:103AF200B1FD9BCDB2FD9CCDB3FD6F0E0D01B46F38
:103B02000D0EB56FA0CDB6FDA1CDB7FD19EC11F02C
:023B120012009F
:103B14004AEC14F08B804AEC14F08B904AEC14F0CD
:103B24008B804AEC14F0100E0D01E66F000EE76F67
:103B3400E86BE96BA2EC00F0110E0D01E66F000ECC
:103B4400E76FE86BE96BA2EC00F0120E0D01E66F73
:103B5400000EE76FE86BE96BA2EC00F0130E0D01A9
:103B6400E66F000EE76FE86BE96BA2EC00F0140E51
:103B74000D01E66F000EE76FE86BE96BA2EC00F055
:103B84000B0E0B6E260E0C6E5D0E0D6E0D2EFED7FB
:103B94000C2EFCD70B2EFAD700000000110E0D01DD
:103BA400E66F000EE76F180EE86F000EE96FA2ECE7
:103BB40000F0120E0D01E66F000EE76F210EE86FA4
:103BC400610EE96FA2EC00F0130E0D01E66F000E1A
:103BD400E76F6F0EE86F000EE96FA2EC00F0140EB1
:103BE4000D01E66F000EE76F5F0EE86F490EE96F97
:103BF400A2EC00F0100E0D01E66F000EE76F000E50
:103C0400E86F080EE96FA2EC00F00B0E0B6E260EA7
:103C14000C6E5D0E0D6E0D2EFED70C2EFCD70B2EEA
:103C2400FAD700000000110E0D01E66F000EE76FD9
:103C34003B0EE86F100EE96FA2EC00F00B0E0B6E5A
:103C4400260E0C6E5D0E0D6E0D2EFED70C2EFCD7BF
:103C54000B2EFAD700000000010E0D01E66F000ED6
:103C6400E76F1C0EE86F010EE96FA2EC00F0020E84
:103C74000D01E66F000EE76F000EE86F010EE96FAD
:103C8400A2EC00F0030E0D01E66F000EE76F300E9C
:103C9400E86F100EE96FA2EC00F0070E0D01E66F5D
:103CA400000EE76FE86BE96BA2EC00F0080E0D0163
:103CB400E66F000EE76F080EE86F080EE96FA2ECDE
:103CC40000F00B0E0D01E66F000EE76F000EE86FBB
:103CD400110EE96FA2EC00F00C0E0D01E66F000E60
:103CE400E76FE86BE96BA2EC00F00F0E0D01E66FD5
:103CF400000EE76F010EE86F0D0EE96FA2EC00F005
:103D0400150E0D01E66F000EE76F200EE86F000E32
:103D1400E96FA2EC00F0200E0D01E66F000EE76FD4
:103D2400E86BE96BA2EC00F0210E0D01E66F000ECA
:103D3400E76FE86BE96BA2EC00F0300E0D01E66F63
:103D4400000EE76FE86BE96BA2EC00F0310E0D0199
:103D5400E66F000EE76FDB0EE86F000EE96FA2EC72
:103D640000F0320E0D01E66F000EE76FE86BE96BB1
:103D7400A2EC00F0330E0D01E66F000EE76FE86B66
:103D8400E96BA2EC00F0340E0D01E66F000EE76F54
:103D9400DB0EE86F000EE96FA2EC00F0350E0D01AA
:103DA400E66F000EE76FE86BE96BA2EC00F0360EED
:103DB4000D01E66F000EE76FAF0EE86F000EE96FBE
:103DC400A2EC00F0370E0D01E66F000EE76FE86B12
:103DD400E96BA2EC00F0380E0D01E66F000EE76F00
:103DE400DB0EE86F000EE96FA2EC00F0390E0D0156
:103DF400E66F000EE76FE86BE96BA2EC00F0500E83
:103E04000D01E66F000EE76FE86BE96BA2EC00F0C2
:103E1400510E0D01E66F000EE76F080EE86F080EF5
:103E2400E96FA2EC00F0520E0D01E66F000EE76F91
:103E34000A0EE86F080EE96FA2EC00F0530E0D01B4
:103E4400E66F000EE76F0A0EE86F000EE96FA2EC52
:103E540000F0540E0D01E66F000EE76F080EE86FD8
:103E64000A0EE96FA2EC00F0550E0D01E66F000E8C
:103E7400E76F080EE86F080EE96FA2EC00F0560E2B
:103E84000D01E66F000EE76FE86BE96BA2EC00F042
:103E9400570E0D01E66F000EE76F000EE86F0A0E75
:103EA400E96FA2EC00F0580E0D01E66F000EE76F0B
:103EB400100EE86F070EE96FA2EC00F0590E0D0129
:103EC400E66F000EE76F100EE86F070EE96FA2ECC5
:103ED40000F0070E0D01E66F000EE76F120EE86F9B
:103EE400000EE96FA2EC00F00B0E0B6E260E0C6EAA
:103EF4005D0E0D6E0D2EFED70C2EFCD70B2EFAD7B1
:103F040000000000070E0D01E66F000EE76F170EAC
:103F1400E86F100EE96FA2EC00F0010E0D01B06F16
:103F240044EC16F0B06B06EC16F00B0E0B6E260E7E
:103F34000C6E5D0E0D6E0D2EFED70C2EFCD70B2EC7
:103F4400FAD700000000B06BB16BA2EC14F00B0EBA
:103F54000B6E260E0C6E5D0E0D6E0D2EFED70C2E06
:103F6400FCD70B2EFAD700000000B06BB16BB26B1C
:103F7400B36BAF0EB46F000EB56FDB0EB66F000EF1
:103F8400B76FB86BB96B2CEC0CF00B0E0B6E260EE6
:103F94000C6E5D0E0D6E0D2EFED70C2EFCD70B2E67
:083FA400FAD700000000120032
:103FAC0057C199FD0D01B06B06EC16F0B06BB16BFF
:103FBC00B26BB36BAF0EB46F000EB56FDB0EB66F9A
:103FCC00000EB76FB86BB96B2CEC0CF099CDB0FD43
:103FDC0006EC16F0680E0C6EE40E0D6E0D2EFED770
:083FEC000C2EFCD700001200AE
:103FF400940E0D01C66FAB0EC76F000EC86F94EC24
:1040040003F0FAD05D0E0D01C66FAB0EC76F000E44
:10401400C86F94EC03F0A50E0D016D6F020E6E6F68
:1040240053C1B0FD54C1B1FD6DCDB2FD6ECDB3FD34
:10403400D1EC12F026D18E0E0D01C66FAA0EC76FF9
:10404400000EC86F94EC03F0650E0D016D6F090E40
:104054006E6F53C1B0FD54C1B1FD6DCDB2FD6ECDD7
:10406400B3FDD1EC12F00DD1100E0D01C66FA90EE7
:10407400C76F000EC86F94EC03F0150E0D016D6F41
:10408400040E6E6F53C1B0FD54C1B1FD6DCDB2FDD0
:104094006ECDB3FDD1EC12F0F4D0920E0D01C66FCB
:1040A400A90EC76F000EC86F94EC03F0250E0D0126
:1040B4006D6F040E6E6F53C1B0FD54C1B1FD6DCD73
:1040C400B2FD6ECDB3FDD1EC12F0DBD0950E0D0137
:1040D400C66FA80EC76F000EC86F94EC03F0FF0EF6
:1040E4000D016D6F040E6E6F53C1B0FD54C1B1FD6F
:1040F4006DCDB2FD6ECDB3FDD1EC12F0C2D0800E09
:104104000D01C66FA80EC76F000EC86F94EC03F0C4
:104114000F0E0D016D6F090E6E6F53C1B0FD54C1CA
:10412400B1FD6DCDB2FD6ECDB3FDD1EC12F0A9D0D1
:10413400EA0E0D01C66FAA0EC76F000EC86F94EC8D
:1041440003F00F0E0D016D6F090E6E6F53C1B0FDBC
:1041540054C1B1FD6DCDB2FD6ECDB3FDD1EC12F005
:1041640090D0330E0D01C66FAB0EC76F000EC86F33
:1041740094EC03F0AC0E0D016D6F060E6E6F53C11F
:10418400B0FD54C1B1FD6DCDB2FD6ECDB3FDD1EC2A
:1041940012F077D06E0E0D01C66FA70EC76F000E1A
:1041A400C86F94EC03F02D0E0D016D6F0A0E6E6F47
:1041B40053C1B0FD54C1B1FD6DCDB2FD6ECDB3FDA3
:1041C400D1EC12F05ED0540E0D01C66FA80EC76F6D
:1041D400000EC86F94EC03F0310E0D016D6F090EE3
:1041E4006E6F53C1B0FD54C1B1FD6DCDB2FD6ECD46
:1041F400B3FDD1EC12F045D0000E0D019A1902E185
:10420400010E9919D8B4FED6000E9A1902E1020ED5
:104214009919D8B410D7000E9A1902E1030E99190E
:10422400D8B422D7000E9A1902E1040E9919D8B411
:1042340034D7000E9A1902E1050E9919D8B446D75D
:10424400000E9A1902E1060E9919D8B458D7000E37
:104254009A1902E1070E9919D8B46AD7000E9A196F
:1042640002E1080E9919D8B47CD7000E9A1902E11C
:10427400090E99198FE0000E9A1902E10A0E991994
:08428400A2E01BEC0CF012009B
:10428C000D019B5101089E6F9F6B000E9F5B010EF1
:10429C00A46F000EA56FFE0E006EFF0E016E9BCD7F
:1042AC0004F0000E056E4FEC02F000C0A0FD01C042
:1042BC00A1FDA66BA76B9BCDA2FD000EA36F800E7C
:1042CC00A719006E800EA319005C02E1A251A65D35
:1042DC00D8B0A0D0800E9F19006E800E005C02E159
:1042EC00000E9E5D0CE3010EA25F000EA35B020E9E
:1042FC00A027000EA123A0519E27A1519F23A64BBE
:10430C00A72B020EA427000EA523A4519E27A5516E
:10431C009F239951A625B06F000EA721B16F9A511A
:10432C00A225B26F000EA321B36FA651995DB46F95
:10433C00A7CDB5FD000EB5579A51A225B66F000E4C
:10434C00A321B76F9CCDB8FD9DCDB9FD33EC15F015
:10435C009951A625B06F000EA721B16FA2519A5D9D
:10436C00B26FA3CDB3FD000EB357A651995DB46FD8
:10437C00A7CDB5FD000EB557A2519A5DB66FA3CD72
:10438C00B7FD000EB7579CCDB8FD9DCDB9FD33ECF4
:10439C0015F09951A225B06F000EA321B16FA65153
:1043AC009A5DB26FA7CDB3FD000EB3579951A225FC
:1043BC00B46F000EA321B56F9A51A625B66F000EEF
:1043CC00A721B76F9CCDB8FD9DCDB9FD33EC15F091
:1043DC00A251995DB06FA3CDB1FD000EB157A6519E
:1043EC009A5DB26FA7CDB3FD000EB357A251995D84
:1043FC00B46FA3CDB5FD000EB5579A51A625B66F77
:10440C00000EA721B76F9CCDB8FD9DCDB9FD33EC47
:10441C0015F055D7A651995DB06FA7CDB1FD000E23
:10442C00B157A2519A5DB26FA3CDB3FD000EB35735
:10443C009951A625B46F000EA721B56F9A51A225EC
:10444C00B66F000EA321B76F9CCDB8FD9DCDB9FD05
:06445C002CEC0CF0120034
:1044620099CDB0FD9ACDB1FD0D01B26BB36B70EC7D
:044472000CF0120038
:104476008B9499CDB0FD9ACDB1FD9BCDB2FD9CCD6F
:10448600B3FD99CDB4FD9ACDB5FD9FCDB6FDA0CDBA
:10449600B7FDA1CDB8FDA2CDB9FD33EC15F099CD90
:1044A600B0FD9ACDB1FD9BCDB2FD9CCDB3FD9DCDAA
:1044B600B4FD9ECDB5FD9BCDB6FD9CCDB7FDA1CD82
:1044C600B8FDA2CDB9FD33EC15F099CDB0FD9ACD6E
:1044D600B1FD9FCDB2FDA0CDB3FD9DCDB4FD9ECD6A
:1044E600B5FD9FCDB6FDA0CDB7FDA1CDB8FDA2CD42
:1044F600B9FD33EC15F09DCDB0FD9ECDB1FD9BCD44
:10450600B2FD9CCDB3FD9DCDB4FD9ECDB5FD9FCD39
:10451600B6FDA0CDB7FDA1CDB8FDA2CDB9FD33EC5A
:0645260015F08B84120069
:10452C000D019D510108A16F9ECDA2FD000EA25759
:10453C00010EA76F000EA86FFE0E006EFF0E016E2F
:10454C009DCD04F09ECD05F04FEC02F000C0A3FD14
:10455C0001C0A4FDA96BAA6B9DCDA5FD9ECDA6FDAA
:10456C0099CDD6FD9ACDD7FD9D519B25D86F9E51E7
:10457C009C21D96F9FCDDAFDA0CDDBFDE1EC01F0E4
:10458C0099CDD6FD9ACDD7FD0D019D519B5DD86F70
:10459C009E519C59D96F9FCDDAFDA0CDDBFDE1EC8E
:1045AC0001F00D019D519925D66F9E519A21D76F1F
:1045BC009BCDD8FD9CCDD9FD9FCDDAFDA0CDDBFDEB
:1045CC00E1EC01F00D019D51995DD66F9E519A5908
:1045DC00D76F9BCDD8FD9CCDD9FD9FCDDAFDA0CD5D
:1045EC00DBFDE1EC01F0800E0D01AA19006E800ECE
:1045FC00A619005C02E1A551A95DD8B0B7D0800E18
:10460C00A219006E800E005C02E1000EA15D0CE3AD
:10461C00010EA55F000EA65B020EA327000EA423BD
:10462C00A351A127A451A223A94BAA2B020EA72761
:10463C00000EA823A751A127A851A223A95199255F
:10464C00D66FAA519A21D76FA5519B25D86FA65129
:10465C009C21D96F9FCDDAFDA0CDDBFDE1EC01F003
:10466C000D01A951995DD66FAA519A59D76FA551D1
:10467C009B25D86FA6519C21D96F9FCDDAFDA0CD7B
:10468C00DBFDE1EC01F00D01A9519925D66FAA5182
:10469C009A21D76FA5519B5DD86FA6519C59D96FA4
:1046AC009FCDDAFDA0CDDBFDE1EC01F00D01A951B0
:1046BC00995DD66FAA519A59D76FA5519B5DD86F4A
:1046CC00A6519C59D96F9FCDDAFDA0CDDBFDE1EC55
:1046DC0001F00D01A5519925D66FA6519A21D76FDE
:1046EC00A9519B25D86FAA519C21D96F9FCDDAFD7A
:1046FC00A0CDDBFDE1EC01F00D01A551995DD66F6C
:10470C00A6519A59D76FA9519B25D86FAA519C21B4
:10471C00D96F9FCDDAFDA0CDDBFDE1EC01F00D01F1
:10472C00A5519925D66FA6519A21D76FA9519B5D9A
:10473C00D86FAA519C59D96F9FCDDAFDA0CDDBFD66
:10474C00E1EC01F00D01A551995DD66FA6519A5976
:10475C00D76FA9519B5DD86FAA519C59D96F9FCD2A
:0E476C00DAFDA0CDDBFDE1EC01F03DD712003F
:10477A00E50E0001F76F0B0EF86F800EF56F010E54
:10478A00F66F010E0D01996F800E006E800E000A01
:10479A00005C02E1140E995D2CE2040E006E000E1C
:1047AA00016E99CD04F0000E056E4FEC02F0F50E85
:1047BA000026000E012200C0E1FF01C0E2FFE66A06
:1047CA00E66A040E006E000E016E99CD04F0000E2A
:1047DA00056E4FEC02F0F50E0026000E0122020EC5
:1047EA000024E16E000E0120E26EE66AE66A992B69
:1047FA00CBD7010E0001E36FE46B01014D6B120090
:10480A000001E45303E0006A016A2BD00D01996BA1
:10481A009A6B9B6B800E006E800E000A005C02E1B0
:10482A00140E9B5D1AE2040E006E000E016E9BCD03
:10483A0004F0000E056E4FEC02F0F50E0026000E95
:10484A000122020E0024D96E000E0120DA6EDE501B
:10485A009927DE509A239B2BDDD799CD00F09ACD6C
:04486A0001F0120047
:10486E0099CDF6FF9ACDF7FF9BCDF8FF0900F5CF56
:10487E0000F0005212E099CDF6FF9ACDF7FF9BCDD6
:10488E00F8FF0900F5CFD6FDCBEC01F0010E0D01BE
:0C489E009927000E9A239B23E3D71200F9
:1048AA00C69AFF0E0001DB6FFF0EDC6FFF0EDD6F95
:1048BA00FF0EDE6F320EDF6F010EE06FEA0EE16F60
:1048CA000D0EE26F949A94969488C66A400EC76E4B
:0448DA00C68A120078
:1048DE000D019F6BA06B000EA05D02E10A0E9F5DA5
:1048EE000BE29F519D25E16EA0519E21E26E200E9E
:1048FE00E66E9F4BA02BEFD79F519D25E16EA051E9
:10490E009E21E26EE66A010E9F5F000EA05B9F5134
:10491E009D25A16FA0519E21A26F0A0E046E000E5E
:10492E00056E066E076E99CD00F09ACD01F09BCD07
:10493E0002F09CCD03F05BEC11F008C000F009C052
:10494E0001F00AC002F00BC003F0300E0026A1CD1C
:10495E00E1FFA2CDE2FF00C0E6FF0A0E046E000EDC
:10496E00056E066E076E99CD00F09ACD01F09BCDC7
:10497E0002F09CCD03F05BEC11F000C099FD01C07C
:10498E009AFD02C09BFD03C09CFD000E046E031831
:10499E0008E10450021805E10450011802E100502C
:1049AE00000A01E105D0010E9F5F000EA05BAFD79C
:0249BE001200E5
:0A49C00033C000F034C001F0120013
:0A49CA0097CD00F098CD01F0120027
:1049D4000001E45303E0006A016A4ED001014D5323
:1049E40002E0ADEC07F00D01996B9A6B9B6B800EA6
:1049F400006E800E000A005C02E1140E9B5D38E23A
:104A0400040E006E000E016E9BCD04F0000E056EC8
:104A14004FEC02F0F50E0026000E0122020E0024D7
:104A2400E96E000E0120EA6EEECF01F0EECF02F047
:104A340002509A5D02E10150995D18E2040E006E85
:104A4400000E016E9BCD04F0000E056E4FEC02F0DB
:104A5400F50E0026000E0122020E0024E96E000E5F
:104A64000120EA6EEECF99FDEECF9AFD9B2BBFD7C6
:0A4A740099CD00F09ACD01F0120078
:104A7E0099CD01F00132019E0132019E0132019E5B
:104A8E000B0E006E01C004F0000E056E005005E026
:104A9E00043604900536FF0FFAD79ACD03F0033291
:104AAE00039E0332039E050E026E03C000F0000E3D
:104ABE00016E025005E0003600900136FF0FFAD766
:104ACE0000500410026E05500110036E9BCD00F0D5
:104ADE000032009E0032009E0032009E000E016EDB
:0A4AEE0002500012035001121200E2
:104AF800FEEC55F0600ED36E9B6A9B8C030E0F0183
:104B0800386F396B3A6BFF0E936E900E946E0F0EE2
:104B1800926EF19E929889983B6A00018B6B0D0109
:104B28006F6B0101586B376A386A396A3A6A2C6ABE
:104B38002D6A226A236A22C020F023C021F03B0E8E
:104B48001C6E000E1D6EDBEC18F0010E0D01996F46
:104B580068EC16F000C01EF001C01FF0B886010E08
:104B6800B06EA00EAF6EAC84A3EC16F0FF0E0D0174
:104B7800996FFF0E9A6F000E9B6F000E9C6F960E3A
:104B88009D6F030E9E6FD60E9F6F0D0EA06FFF0ECA
:104B9800A16FFF0EA26F000EA36F000EA46FFF0E91
:104BA800A56FFF0EA66F000EA76F000EA86F47EC4B
:104BB80016F0090E0B6E1E0E0C6EE40E0D6E0D2E09
:104BC800FED70C2EFCD70B2EFAD700000C0ED66F92
:104BD800CBEC01F01BEC0CF04D0E0D01C66FAA0ECC
:104BE800C76F000EC86F94EC03F0410E0D01C66F3D
:104BF800A60EC76F000EC86F94EC03F0F20E0D01FD
:104C0800C66FA30EC76F000EC86F94EC03F0810E39
:104C18000D01C66FA40EC76F000EC86F94EC03F0A9
:104C2800BB0E0D01C66FA30EC76F000EC86F94ECC4
:104C380003F01A0E0D01C66FAA0EC76F000EC86FDB
:104C480094EC03F01BEC0CF0090E0B6E1E0E0C6EB0
:104C5800E40E0D6E0D2EFED70C2EFCD70B2EFAD7B8
:104C68000000376A386A396A3A6A2C6A2D6A000E77
:104C7800231802E1000E2218010ED8A4000E206E9F
:104C8800000E216ED08EF28C9D9AF29E2A6A2B6AB3
:104C98000101556B566B196A240E0D01C66FA40EDF
:104CA800C76F000EC86F94EC03F0EEEC18F02FC03D
:104CB80099FD30C09AFD31C09BFD32C09CFD580E55
:104CC8009D6F010E9E6F020E9F6FD7EC16F0410E7E
:104CD800996FAB0E9A6F000E9B6FC5DD580E0D01D4
:104CE800C66F010EC76FC5EC05F0E10E996FAB0EEC
:104CF8009A6F000E9B6FB7DD4F0E0D01C66FAB0E9E
:104D0800C76F000EC86F94EC03F0CBDDB60E0D0133
:104D1800996FA70E9A6F000E9B6FA5DD2ADD71DDD6
:104D280000C024F001C025F0000E266E276E24C0B6
:104D380099FD25C09AFD26C09BFD27C09CFD580EF5
:104D48000D019D6F010E9E6FC6DD800E996FA90E35
:104D58009A6F000E9B6F87DD580E0D01C66F010E0E
:104D6800C76FC5EC05F01BEC0CF030DE00C024F07A
:104D780001C025F0000E266E276E24C099FD25C0BF
:104D88009AFD26C09BFD27C09CFD580E0D019D6F06
:104D9800010E9E6FA0DDA90E996FA60E9A6F000EE8
:104DA8009B6F61DD580E0D01C66F010EC76FC5EC14
:104DB80005F01BEC0CF0AE0E0D01996FA40E9A6F66
:104DC800000E9B6F50DD080E0D01C66FA60EC76F53
:104DD800000EC86F94EC03F04AEC14F0FF0E0D01BE
:104DE800996FFF0E9A6F9B6B46DE00C028F001C0DA
:104DF80029F00D01B06B06EC16F0DEDD00C049F1BC
:104E080001C04AF149C1B0FD4AC1B1FD580EB26FA7
:104E1800010EB36F57EC14F0F30E996FAB0E9A6F47
:104E2800000E9B6F20DD580E0D01C66F010EC76F77
:104E3800C5EC05F0C6DD00C049F101C04AF149C121
:104E4800B0FD4AC1B1FD580EB26F010EB36F57ECF9
:104E580014F0DA0E996FAB0E9A6F000E9B6F03DD9C
:104E6800580E0D01C66F010EC76FC5EC05F01BEC9F
:104E78000CF00D01B06BB16BA2EC14F0DE6BDF6BC4
:104E8800E06BE16BAF0EE26F000EE36FDB0EE46FD9
:104E9800000EE56F1FEC01F08AEC1DF0B06BB16BF2
:104EA800A2EC14F0FF0E996FFF0E9A6F9B6BE3DD77
:104EB80000C028F001C029F00D01B06BB16BB26BD6
:104EC800B36BAF0EB46F000EB56FDB0EB66F000E8E
:104ED800B76FB86BB96B2CEC0CF0B06BB16BA2EC84
:104EE80014F0996BFF0E9A6F9B6BC5DD00C028F01C
:104EF80001C029F00D01DE6BDF6BE06BE16BAF0EDB
:104F0800E26F000EE36FDB0EE46F000EE56F1FEC3F
:104F180001F0AD0E0D01C66FAB0EC76F000EC86F66
:104F280094EC03F0D6EC1FF01BEC0CF01BEC0CF02F
:104F3800260E0D01C66FA70EC76F000EC86F94EC42
:104F480003F0D6EC1FF0010E01014B6F000E4C6F01
:104F58004BC199FD4CC19AFD93EC19F0010E0D015E
:104F6800996F000E9A6F010E9B6F000E9C6F8F0E4B
:104F78009D6FA60E9E6F000E9F6FFF0EA06F070E0F
:104F8800A16F69EC1DF06F0EB06F0D0EB16F260E9C
:104F9800B26FA60EB36F000EB46FBFEC0EF0010E29
:104FA8000D01B06F000EB16FB40EB26F000EB36F8B
:104FB8006F0EB46F0D0EB56FFF0EB66F070EB76F9D
:104FC80019EC11F0100E996F000E9A6F160E9B6F68
:104FD800000E9C6F870E9D6FAB0E9E6F000E9F6F2D
:104FE800E00EA06FFF0EA16F69EC1DF0020E996F25
:104FF800000E9A6F200E9B6F000E9C6FDB0E9D6F4C
:10500800A60E9E6F000E9F6FFF0EA06FFF0EA16F82
:1050180069EC1DF0020E996F000E9A6F2A0E9B6FB5
:10502800000E9C6FBD0E9D6FAA0E9E6F000E9F6FA7
:10503800FF0EA06F070EA16F69EC1DF0020E996FAD
:10504800000E9A6F340E9B6F000E9C6F9E0E9D6F24
:10505800A70E9E6F000E9F6FFF0EA06F070EA16F29
:1050680069EC1DF0020E996F000E9A6F3E0E9B6F51
:10507800000E9C6FDA0E9D6FA40E9E6F000E9F6F40
:10508800FF0EA06F070EA16F69EC1DF0020E996F5D
:10509800000E9A6F480E9B6F000E9C6F210E9D6F3D
:1050A800A50E9E6F000E9F6FFF0EA06F070EA16FDB
:1050B80069EC1DF0020E996F000E9A6F520E9B6FED
:1050C800000E9C6FA10E9D6FAB0E9E6F000E9F6F22
:1050D800E00EA06F070EA16F69EC1DF0020E996F2C
:1050E800000E9A6F5C0E9B6F000E9C6FFE0E9D6FFC
:1050F800A40E9E6F000E9F6FFF0EA06F070EA16F8C
:1051080069EC1DF0020E996F000E9A6F660E9B6F88
:10511800000E9C6F3C0E9D6FAA0E9E6F000E9F6F37
:10512800FF0EA06F070EA16F69EC1DF0020E996FBC
:10513800000E9A6F700E9B6F000E9C6F6A0E9D6F2B
:10514800A80E9E6F000E9F6FFF0EA06F070EA16F37
:1051580069EC1DF0020E996F000E9A6F840E9B6F1A
:10516800000E9C6F4A0E9D6FA90E9E6F000E9F6FDA
:105178001F0EA06FF80EA16F69EC1DF04AEC14F039
:105188004AEC14F0D6EC1FF0240EC66FA90EC76FB8
:10519800000EC86F94EC03F06F0E0D01B06F0D0E8A
:1051A800B16F9E0EB26FAA0EB36F000EB46FBFEC54
:1051B8000EF0200E0D01B06F000EB16F200EB26F11
:1051C800000EB36F6F0EB46F0D0EB56FE00EB66FB5
:1051D800070EB76F19EC11F04BC199FD4CC19AFD40
:1051E800FAEC1FF04AEC14F0870E0D01C66FA50EFD
:1051F800C76F000EC86F94EC03F00D01B06BB16B74
:10520800B26BB36BAF0EB46F000EB56FB66BB76B06
:105218001D0EB86FEC0EB96F33EC15F0B06BB16BB7
:10522800DB0EB26F000EB36FAF0EB46F000EB56F2A
:10523800DB0EB66F000EB76F1D0EB86FEC0EB96FB0
:1052480033EC15F0B06BB16BB26BB36BAF0EB46FE0
:10525800000EB56FDB0EB66F000EB76F1D0EB86F80
:10526800EC0EB96F33EC15F0AF0EB06F000EB16FE6
:10527800B26BB36BAF0EB46F000EB56FDB0EB66FCB
:10528800000EB76F1D0EB86FEC0EB96F33EC15F04A
:10529800C50EC66FA90EC76F000EC86F94EC03F059
:1052A800010E0D01B06F000EB16F010EB26F000E4E
:1052B800B36FAF0EB46F000EB56FDB0EB66F000E96
:1052C800B76FE00EB86F070EB96F33EC15F0A80E84
:1052D800C66FA50EC76F000EC86F94EC03F0010EE1
:1052E8000D01B06F000EB16F640EB26F000EB36F98
:1052F800AF0EB46F000EB56F640EB66F000EB76FC9
:10530800000EB86FF80EB96F33EC15F04AEC14F0D4
:10531800650EC66FA50EC76F000EC86F94EC03F03C
:105328000101556B566B800E5619006E800E005C9D
:1053380002E1DB0E555D13E2500E0D01D66F000E33
:10534800D76F55C1D8FD56C1D9FDE00EDA6FFF0EF3
:10535800DB6FE1EC01F00101554B562BE4D7C90E88
:105368000D01C66FA50EC76F000EC86F94EC03F051
:105378005A0E0D01B06F000EB16F010EB26F000E24
:10538800B36F5A0EB46F000EB56FDB0EB66F000E1A
:10539800B76F450EB86FA10EB96F33EC15F0010E5B
:1053A800B06F000EB16F010EB26F000EB36F010E39
:1053B800B46F000EB56FDA0EB66F000EB76FFF0E42
:1053C800B86FFF0EB96F33EC15F0AE0EB06F000E6C
:1053D800B16F020EB26F000EB36FAE0EB46F000E57
:1053E800B56FDA0EB66F000EB76FFF0EB86FFF0E0F
:1053F800B96F33EC15F04AEC14F0A30EC66FA90E82
:10540800C76F000EC86F94EC03F0010E0D01B06F6A
:10541800000EB16FDB0EB26F000EB36FAF0EB46F3C
:10542800000EB56F010EB66F000EB76F1F0EB86F86
:10543800000EB96F33EC15F05C0EC66FA90EC76F7E
:10544800000EC86F94EC03F0180E0D01996F000E52
:105458009A6F180E9B6F000E9C6F440E9D6F000E86
:105468009E6F600E9F6F000EA06FFF0EA16FFF0E64
:10547800A26F3BEC22F04AEC14F0F80EC66FA90EAE
:10548800C76F000EC86F94EC03F0200E0D01996FE2
:10549800000E9A6F300E9B6F000E9C6F100E9D6F62
:1054A800000E9E6F1F0E9F6FF80EA06F96EC22F0F5
:1054B8004AEC14F05E0E0D01C66FAA0EC76F000EFF
:1054C800C86F94EC03F0240E0D01996F000E9A6FCB
:1054D800340E9B6F000E9C6F100E9D6F000E9E6F1A
:1054E800FF0E9F6FFF0EA06F96EC22F04AEC14F0AF
:1054F800D40E0D01C66FA80EC76F000EC86F94ECCE
:1055080003F0300E0D01996F780E9A6F100E9B6F95
:10551800A00E9C6FFE0E9D6F46EC21F04AEC14F035
:105528003E0EC66FA70EC76F000EC86F94EC03F04F
:10553800560E0D01B06F000EB16F560EB26F000E11
:10554800B36F800EB46F000EB56F800EB66F000E8D
:10555800B76FE00EB86FFF0EB96F2CEC0CF04AEC89
:1055680014F0E40EC66FA70EC76F000EC86F94EC58
:1055780003F0640E0D01B06F000EB16F100EB26F24
:10558800000EB36FA00EB46F000EB56F200EB66F8D
:10559800000EB76FFF0EB86F070EB96F2CEC0CF04A
:1055A8004AEC14F0CC0EC66FAA0EC76F000EC86F77
:1055B80094EC03F0400E0D01996F000E9A6F8C0E5B
:1055C8009B6F000E9C6F140E9D6F000E9E6FE00E79
:1055D8009F6FFF0EA06F96EC22F04AEC14F0790E44
:1055E8000D01C66FAB0EC76F000EC86F94EC03F0C9
:1055F800910E0D01996F000E9A6FB90E9B6F000EF8
:105608009C6F1E0E9D6F000E9E6FE00E9F6F070E23
:10561800A06F96EC22F04AEC14F03E0E0D01C66F16
:10562800A80EC76F000EC86F94EC03F04AEC14F094
:105638004AEC14F0D6EC1FF0000E231802E1000E1D
:105648002218010ED8A4000E206E000E216ED08EF6
:10565800F28C9D8AF28E2A6A2B6A140E2F6EAE0E79
:10566800306ECF0E316E820E326E010E01014B6F1D
:10567800000E4C6F4BC199FD4CC19AFD93EC19F08B
:105688006F0E0D01B06F0D0EB16F370EB26FA90E10
:10569800B36F000EB46FBFEC0EF0010E0D01B06FCA
:1056A800000EB16F640EB26F000EB36F6F0EB46F61
:1056B8000D0EB56FE00EB66F070EB76F19EC11F04F
:1056C8006F0EC66F0D0EC76FC5EC05F01BEC0CF026
:1056D8004BC199FD4CC19AFDFAEC1FF01BEC0CF084
:1056E800020E01014B6F000E4C6F4BC199FD4CC16E
:1056F8009AFD93EC19F0430E0D01C66FA50EC76F06
:10570800000EC86F94EC03F0010E0D01996F000EA6
:105718009A6F100E9B6F000E9C6FAE0E9D6FAA0EB7
:105728009E6F000E9F6FE00EA06FFF0EA16F69ECD9
:105738001DF0120E996FA80E9A6F000E9B6F37EC32
:1057480024F04BC199FD4CC19AFDFAEC1FF01BECFB
:105758000CF04AEC14F04AEC14F01A50010A02E179
:10576800EEEC18F0030E01014B6F000E4C6F4BC1AD
:1057780099FD4CC19AFD93EC19F0530E0D01C66FBB
:10578800A40EC76F000EC86F94EC03F06F0E0D01E6
:10579800B06F0D0EB16F6E0EB26FA90EB36F000E23
:1057A800B46FBFEC0EF06F0E0D01C66F0D0EC76F14
:1057B80063EC0BF000C049F101C04AF1010EB06F73
:1057C800000EB16F460EB26F000EB36F6F0EB46F5E
:1057D8000D0EB56F1F0EB66FF80EB76F19EC11F0FE
:1057E8002FC099FD30C09AFD31C09BFD32C09CFD91
:1057F800580E9D6F010E9E6F020E9F6FD7EC16F02C
:10580800090E996FAA0E9A6F000E9B6F37EC24F061
:10581800580E0D01C66F010EC76FC5EC05F0E70EF7
:10582800996FAB0E9A6F000E9B6F37EC24F02FC068
:1058380000F030C001F031C002F032C003F045C1C1
:1058480004F046C105F047C106F048C107F04CEC2A
:105858000BF0000ED8A4010E006E005213E0010EEA
:105868000D01996F000E9A6F0A0E9B6F000E9C6FC8
:10587800C20E9D6FAB0E9E6F000E9F6FA06BA16B4B
:1058880069EC1DF00D01010EB06F000EB16F6E0EC8
:10589800B26F000EB36F580EB46F010EB56FFF0EE6
:1058A800B66FFF0EB76F19EC11F0580EC66F010EE8
:1058B800C76FC5EC05F04BC199FD4CC19AFDFAECD8
:1058C8001FF0040E01014B6F000E4C6F4BC199FD88
:1058D8004CC19AFD93EC19F0C20E0D01C66FA60ECD
:1058E800C76F000EC86F94EC03F0580E0D01B06F2F
:1058F800010EB16FE90EB26FA50EB36F000EB46F53
:10590800BFEC0EF00D01B06BB16B280EB26F000E3C
:10591800B36F580EB46F010EB56FFF0EB66F070E5A
:10592800B76F19EC11F0580EC66F010EC76FC5ECB2
:1059380005F04BC199FD4CC19AFDFAEC1FF0050E1C
:1059480001014B6F000E4C6F4BC199FD4CC19AFD84
:1059580093EC19F0750E0D01C66FA60EC76F000EF9
:10596800C86F94EC03F02FC099FD30C09AFD31C088
:105978009BFD32C09CFD580E0D019D6F010E9E6F60
:10598800020E9F6FD7EC16F0B40E996FA90E9A6F9E
:10599800000E9B6F37EC24F0580E0D01C66F010EF8
:1059A800C76FC5EC05F0ED0E996FAB0E9A6F000E40
:1059B8009B6F37EC24F02FC000F030C001F031C0ED
:1059C80002F032C003F045C104F046C105F047C1FA
:1059D80006F048C107F04CEC0BF0000ED8A4010EFD
:1059E800006E005213E0010E0D01996F000E9A6FC0
:1059F8008C0E9B6F000E9C6FD20E9D6FAB0E9E6F30
:105A0800000E9F6FA06BA16B69EC1DF00D01010EDC
:105A1800B06F000EB16F8C0EB26F000EB36F580EE0
:105A2800B46F010EB56F200EB66FFD0EB76F19EC8F
:105A380011F04BC199FD4CC19AFDFAEC1FF04AECEC
:105A480014F04AEC14F0D6EC1FF0010E01014B6F74
:105A5800000E4C6F4BC199FD4CC19AFD93EC19F0A7
:105A68006F0E0D01B06F0D0EB16F860EB26FA70EDF
:105A7800B36F000EB46FBFEC0EF0010E0D01B06FE6
:105A8800000EB16F870EB26F000EB36F6F0EB46F5A
:105A98000D0EB56F1F0EB66FF80EB76F19EC11F03B
:105AA8004BC199FD4CC19AFDFAEC1FF0060E01019D
:105AB8004B6F000E4C6F4BC199FD4CC19AFD93EC96
:105AC80019F05B0E0D01C66FA60EC76F000EC86FEA
:105AD80094EC03F02FC099FD30C09AFD31C09BFDB6
:105AE80032C09CFD580E0D019D6F010E9E6F020E77
:105AF8009F6FD7EC16F0010EB06F000EB16F910ECC
:105B0800B26F000EB36F580EB46F010EB56F1F0E53
:105B1800B66F000EB76F19EC11F04BC199FD4CC16F
:105B28009AFDFAEC1FF0010E01014B6F000E4C6F4D
:105B38004BC199FD4CC19AFD93EC19F06F0E0D0104
:105B4800B06F0D0EB16FCD0EB26FA70EB36F000E12
:105B5800B46FBFEC0EF0010E0D01B06F000EB16F07
:105B6800140EB26F000EB36F6F0EB46F0D0EB56FDB
:105B7800FF0EB66F070EB76F19EC11F04BC199FD08
:105B88004CC19AFDFAEC1FF0070E01014B6F000E95
:105B98004C6F4BC199FD4CC19AFD93EC19F00D0E59
:105BA8000D01C66FA70EC76F000EC86F94EC03F007
:105BB8002FC099FD30C09AFD31C09BFD32C09CFDBD
:105BC800580E0D019D6F010E9E6F020E9F6FD7EC50
:105BD80016F02FC000F030C001F031C002F032C022
:105BE80003F045C104F046C105F047C106F048C1BD
:105BF80007F04CEC0BF0000ED8A4010E006E00521A
:105C080012E0010E996F000E9A6F280E9B6F000E1E
:105C18009C6FCA0E9D6FAB0E9E6F000E9F6FA06BA0
:105C2800A16B69EC1DF02FC004F030C005F031C045
:105C380006F032C007F0006A016A026A036AC3EC20
:105C48000AF0010ED8B0000E006E005213E0010EEB
:105C5800B06F000EB16F280EB26F000EB36F580E02
:105C6800B46F010EB56F000EB66FF80EB76F19EC72
:105C780011F012D0010EB06F000EB16F280EB26F86
:105C8800000EB36F580EB46F010EB56F1F0EB66FCE
:105C9800000EB76F19EC11F04BC199FD4CC19AFD7C
:105CA800FAEC1FF04AEC14F0010E01014B6F000EE4
:105CB8004C6F4BC199FD4CC19AFD93EC19F06F0ED6
:105CC8000D01B06F0D0EB16FFB0EB26FA70EB36F63
:105CD800000EB46FBFEC0EF0010E0D01B06F000E98
:105CE800B16F500EB26F000EB36F6F0EB46F0D0E22
:105CF800B56FE00EB66FFF0EB76F19EC11F04BC120
:105D080099FD4CC19AFDFAEC1FF0FF0E0D01B06F22
:105D1800FF0EB16FA2EC14F0080E01014B6F000EDC
:105D28004C6F4BC199FD4CC19AFD93EC19F0F40EE0
:105D38000D01C66FA60EC76F000EC86F94EC03F076
:105D48002FC099FD30C09AFD31C09BFD32C09CFD2B
:105D5800580E0D019D6F010E9E6F020E9F6FD7ECBE
:105D680016F0010EB06F000EB16F5F0EB26F000E2D
:105D7800B36F580EB46F010EB56FB66BB76B19ECF5
:105D880011F04BC199FD4CC19AFDFAEC1FF00D01C1
:105D9800B06BB16BA2EC14F04AEC14F04AEC14F0BE
:105DA8002FC045F130C046F131C047F132C048F14B
:105DB8004AEC14F04AEC14F04AEC14F0D6EC1FF05C
:105DC800000E2D1802E1010E2C183AE1B90E996F58
:105DD800AB0E9A6F000E9B6F37EC24F08B0E0D0103
:105DE800C66F000EC76FC5EC05F01BEC0CF0000188
:105DF8008B51540A13E18C513D0A10E18D0E0D01AF
:105E0800996F000E9A6F31EC22F000C02FF001C09C
:105E180030F002C031F003C032F01A6A00018B5131
:105E28004D0A02E1010E1A6E2C6A2D6A8B6B396AD3
:105E38003A6A376A386AAECF4EF101014E6B9D8AD5
:085E48001BEC0CF08AD4FFD71B
:10ABFC0010EE19F0030E006E010E016EF90EF66EDA
:0EAC0C00AB0EF76E000EF86ECFEC16F01200D5
:105E500020322E0D050000000000000000000000B0
:105E60000000000000000000000000000000000032
:105E70000000000000000000000000000000000022
:105E80000000000000000000000000000000000012
:105E90000000000000000000000000000000000002
:105EA00000000000000000000000000000000000F2
:105EB00000000000000000000000000000000000E2
:105EC00000000000000000000000000000000000D2
:105ED00000000000000000000000000000000000C2
:105EE000000000000000000000000000000000E0D2
:105EF000000001F0000003F8000003F8000003F8C0
:105F0000000001F0000000E00000000000000000C0
:105F10000000000000000000000000000000000081
:105F20000000000000000000000000000000000071
:105F30000000000000000000000000000000000061
:105F40000000000000000000000000000000000051
:105F50000000000000000000000000000000000041
:105F60000000000000000000000000000000000031
:105F70000000000000000000000000000000000021
:105F80000000000000000000000000000000000011
:105F90000000000000000000000000000000000001
:105FA00000000000000000000000000000000000F1
:105FB00000000000000000000000000000000000E1
:105FC00000000000000000000000000000000000D1
:105FD00000000000000000000000000000000000C1
:105FE0000000000000000000000000000000FFFEB4
:105FF0000001FFFF0003FFFF8001FFFF600CFFFEB9
:10600000F01E0001F83F0001F83F0001F83F0001D9
:10601000F83F0001F83F0001F83F0001F83F0001A0
:10602000F83F0001F83F0001F83F0001F83F000190
:10603000F83F0001F83F0001F83E0000783800000A
:1060400018200000080000000020000000380000B8
:10605000183E0000783F0001F83F0001F83F0001C2
:10606000F83F0001F83F0001F83F0001F83F000150
:10607000F83F0001F83F0001F83F0001F83F000140
:10608000F83F0001F83F0001F83F0001F81E000052
:10609000F00CFFFE6001FFFF0003FFFF8001FFFF28
:1060A0000000FFFE000000000000000000000000F3
:1060B00000000000000000000000000000000000E0
:1060C0000000000060000000F0000001F800000186
:1060D000F8000001F8000001F8000001F8000001DC
:1060E000F8000001F8000001F8000001F8000001CC
:1060F000F8000001F8000001F8000001F8000001BC
:10610000F8000000780000001800000008000000FF
:1061100000000000000000001800000078000001EE
:10612000F8000001F8000001F8000001F80000018B
:10613000F8000001F8000001F8000001F80000017B
:10614000F8000001F8000001F8000001F80000016B
:10615000F8000001F8000000F000000060000000FE
:10616000000000000000000000000000000000002F
:106170000000000000000000000000000000FFFE22
:106180000001FFFF0003FFFF8001FFFF6000FFFE33
:10619000F0000001F8000001F8000001F800000123
:1061A000F8000001F8000001F8000001F80000010B
:1061B000F8000001F8000001F8000001F8000001FB
:1061C000F8000001F8000001F80000007801FFFE6F
:1061D0001803FFFF880FFFFFE027FFFFC039FFFF15
:1061E000003E0000003F0000003F0000003F0000B4
:1061F000003F0000003F0000003F0000003F0000A3
:10620000003F0000003F0000003F0000003F000092
:10621000003F0000003F0000003F0000001E0000A3
:10622000000CFFFE0001FFFF0003FFFF8001FFFFE6
:106230000000FFFE00000000000000000000000061
:10624000000000000000FFFE0001FFFF0003FFFF51
:106250008001FFFF6000FFFEF0000001F800000178
:10626000F8000001F8000001F8000001F80000014A
:10627000F8000001F8000001F8000001F80000013A
:10628000F8000001F8000001F8000001F80000012A
:10629000F80000007801FFFE1803FFFF880FFFFFE2
:1062A000E007FFFFC001FFFF1800000078000001B9
:1062B000F8000001F8000001F8000001F8000001FA
:1062C000F8000001F8000001F8000001F8000001EA
:1062D000F8000001F8000001F8000001F8000001DA
:1062E000F8000001F8000000F000FFFE6001FFFF71
:1062F0000003FFFF8001FFFF0000FFFE0000000021
:10630000000000000000000000000000000000008D
:10631000000000000000000000000000600C000011
:10632000F01E0001F83F0001F83F0001F83F0001B6
:10633000F83F0001F83F0001F83F0001F83F00017D
:10634000F83F0001F83F0001F83F0001F83F00016D
:10635000F83F0001F83F0001F83E00007839FFFEE9
:106360001823FFFF880FFFFFE007FFFFC001FFFFBB
:106370001800000078000001F8000001F80000019A
:10638000F8000001F8000001F8000001F800000129
:10639000F8000001F8000001F8000001F800000119
:1063A000F8000001F8000001F8000001F80000000A
:1063B000F00000006000000000000000000000008D
:1063C00000000000000000000000000000000000CD
:1063D000000000000000FFFE0001FFFF0003FFFFC0
:1063E0008001FFFF000CFFFE001E0000003F0000C8
:1063F000003F0000003F0000003F0000003F0000A1
:10640000003F0000003F0000003F0000003F000090
:10641000003F0000003F0000003F0000003F000080
:10642000003E00000039FFFE0023FFFF800FFFFF4A
:10643000E007FFFFC001FFFF180000007800000127
:10644000F8000001F8000001F8000001F800000168
:10645000F8000001F8000001F8000001F800000158
:10646000F8000001F8000001F8000001F800000148
:10647000F8000001F8000000F000FFFE6001FFFFDF
:106480000003FFFF8001FFFF0000FFFE000000008F
:106490000000000000000000000000000000FFFEFF
:1064A0000001FFFF0003FFFF8001FFFF000CFFFE64
:1064B000001E0000003F0000003F0000003F000001
:1064C000003F0000003F0000003F0000003F0000D0
:1064D000003F0000003F0000003F0000003F0000C0
:1064E000003F0000003F0000003E00000039FFFEBA
:1064F0000023FFFF800FFFFFE027FFFFC039FFFFF2
:10650000183E0000783F0001F83F0001F83F00010D
:10651000F83F0001F83F0001F83F0001F83F00019B
:10652000F83F0001F83F0001F83F0001F83F00018B
:10653000F83F0001F83F0001F83F0001F81E00009D
:10654000F00CFFFE6001FFFF0003FFFF8001FFFF73
:106550000000FFFE0000000000000000000000003E
:10656000000000000000FFFE0001FFFF0003FFFF2E
:106570008001FFFF6000FFFEF0000001F800000155
:10658000F8000001F8000001F8000001F800000127
:10659000F8000001F8000001F8000001F800000117
:1065A000F8000001F8000001F8000001F800000107
:1065B000F80000007800000018000000080000004B
:1065C000000000000000000018000000780000013A
:1065D000F8000001F8000001F8000001F8000001D7
:1065E000F8000001F8000001F8000001F8000001C7
:1065F000F8000001F8000001F8000001F8000001B7
:10660000F8000001F8000000F00000006000000049
:10661000000000000000000000000000000000007A
:106620000000000000000000000000000000FFFE6D
:106630000001FFFF0003FFFF8001FFFF600CFFFE72
:10664000F01E0001F83F0001F83F0001F83F000193
:10665000F83F0001F83F0001F83F0001F83F00015A
:10666000F83F0001F83F0001F83F0001F83F00014A
:10667000F83F0001F83F0001F83E00007839FFFEC6
:106680001823FFFF880FFFFFE027FFFFC039FFFF40
:10669000183E0000783F0001F83F0001F83F00017C
:1066A000F83F0001F83F0001F83F0001F83F00010A
:1066B000F83F0001F83F0001F83F0001F83F0001FA
:1066C000F83F0001F83F0001F83F0001F81E00000C
:1066D000F00CFFFE6001FFFF0003FFFF8001FFFFE2
:1066E0000000FFFE000000000000000000000000AD
:1066F000000000000000FFFE0001FFFF0003FFFF9D
:106700008001FFFF600CFFFEF01E0001F83F00015A
:10671000F83F0001F83F0001F83F0001F83F000199
:10672000F83F0001F83F0001F83F0001F83F000189
:10673000F83F0001F83F0001F83F0001F83F000179
:10674000F83E00007839FFFE1823FFFF880FFFFF97
:10675000E007FFFFC001FFFF180000007800000104
:10676000F8000001F8000001F8000001F800000145
:10677000F8000001F8000001F8000001F800000135
:10678000F8000001F8000001F8000001F800000125
:10679000F8000001F8000000F000FFFE6001FFFFBC
:1067A0000003FFFF8001FFFF0000FFFE000000006C
:1067B00000000000000000000000000000000000D9
:1067C00000000000000000000000000000000000C9
:1067D00000000000000000000000000000000000B9
:1067E00000000000000000E0000001F0000003F8DD
:1067F000000003F8000003F8000001F0000000E0D2
:106800000000000000000000000000000000000088
:106810000000000000000000000000000000000078
:106820000000000000000000000000000000000068
:106830000000000000000000000000E0000001F087
:10684000000003F8000003F8000003F8000001F066
:10685000000000E000000000000000000000000058
:106860000000000000000000000000000000000028
:0D687000000000000000000000000000001B
:10687D000C1020600E07000000000000000000005A
:10688D0000000000000000000000000000000800F3
:10689D0000000000007C00FF33FF33FF337C00005D
:1068AD000000000000000009000000003C003C005A
:1068BD003C0000003C003C003C00000000000000DB
:1068CD000C0002101E901FF01FFE037E1E9E1FF077
:1068DD001FFE037E021E0010000A00007804FC0C4F
:1068ED00FC0CFF3FFF3FFF3FCC0FCC0F8807000094
:1068FD0000000C00303838383C381E380F8007C087
:10690D0003E039F03878383C381C000B0000001FCC
:10691D00B83FFC3FFE31E637FE3F3E1E1C3E0036C3
:10692D00002200000700000000000027003F003F8C
:10693D00001F000000000000000000000009000022
:10694D000000F003FC0FFE1FFF3F07380120012060
:10695D0000000000000009000000000120012007D8
:10696D0038FF3FFE1FFC0FF0030000000000000A7F
:10697D000000980CB80EF80FF80FF80FF80FF80F7D
:10698D00B80E980C000000000A0000800180018004
:10699D0001F00FF00FF00F80018001800100000069
:1069AD00000700000000000000B800F800F80078B3
:1069BD00000000000000000000000A0000800180BF
:1069CD000180018001800180018001800180010032
:1069DD0000000007000000000000003800380038FB
:1069ED000038000000000000000000000C0018003E
:1069FD001C001E000F8007C003E001F00078003C72
:106A0D00001E000E000CF807FE1FFE1F073F83330C
:106A1D00C331E33073303F38FE1FFE1FF8070B0004
:106A2D000000000C300C300E30FF3FFF3FFF3F00E9
:106A3D00300030003000000C1C301E381F3C073E6B
:106A4D00033F8337C333E331F7307F303E301C30A3
:106A5D000C0C0C0E1C0F3CC738C330C330C330C3F5
:106A6D0030E739FF3F7E1F3C0E0CC003E003F003FF
:106A7D0078033C031E030F03FF3FFF3FFF3F00035F
:106A8D0000030C3F0C7F1C7F3C6338633063306325
:106A9D00306330E338E33FC31F830F0CC00FF01F8B
:106AAD00F83FFC39DE30CF30C730C330C339C33F78
:106ABD00801F000F0C0300030003000330033C0391
:106ACD003FC30FF303FF003F000F0003000C000F47
:106ADD00BC1FFE3FFF39E730C330C330E730FF390D
:106AED00FE3FBC1F000F0C3C007E00FF30E730C3A3
:106AFD0030C338C33CC31EE70FFF07FE03FC00077E
:106B0D00000000000000701C701C701C701C000048
:106B1D0000000000000000000700000000000070F1
:106B2D009C70FC70FC707C000000000000000000F8
:106B3D00000A0000C000E001F003F8073C0F1E1E24
:106B4D000F3C07380330000000000B0000600660AA
:106B5D0006600660066006600660066006600660F8
:106B6D000600000A0000033007380F3C1E1E3C0FC4
:106B7D00F807F003E001C000000000000B1C001E30
:106B8D00001F0007008337C337E337F7007F003E50
:106B9D00001C0000000CF80FFE1FFF1FF73BFB371A
:106BAD00FB37FB37FB37FF37FF37FE03F8010B00D1
:106BBD0038003FE03FFC07FF061F06FF06FC07E01D
:106BCD003F003F003800000BFF3FFF3FFF3FC3304A
:106BDD00C330C330E730FF39FE3FBC1F000F00004C
:106BED000BF003FC0FFE1F0F3C073803300330077B
:106BFD00380F3C0E1C0C0C00000BFF3FFF3FFF3FFE
:106C0D0003300330033007380F3CFE1FFC0FF00339
:106C1D0000000BFF3FFF3FFF3FC330C330C330C306
:106C2D0030C330C3300330033000000BFF3FFF3F54
:106C3D00FF3FC300C300C300C300C300C300030074
:106C4D00030000000BF003FC0FFE1F0F3C0738C3C1
:106C5D0030C330C330C73FC73FC63F00000BFF3FB7
:106C6D00FF3FFF3FC000C000C000C000C000FF3F9D
:106C7D00FF3FFF3F0000090000000003300330FF1D
:106C8D003FFF3FFF3F033003300000000000000BCB
:106C9D00000E001E003E003800300030003000387D
:106CAD00FF3FFF1FFF0700000BFF3FFF3FFF3FE0D0
:106CBD0001F003F8073C0F1E1E0F3C073803300090
:106CCD00000BFF3FFF3FFF3F003000300030003032
:106CDD00003000300030003000000BFF3FFF3FFF61
:106CED003F7E00F801E001F8017E00FF3FFF3FFF0E
:106CFD003F00000BFF3FFF3FFF3F3E00F800F0035A
:106D0D00C007001FFF3FFF3FFF3F00000BF003FCDC
:106D1D000FFE1F0F3C0738033007380F3CFE1FFCDA
:106D2D000FF00300000BFF3FFF3FFF3F8301830187
:106D3D0083018301C701FF01FE007C0000000BF001
:106D4D0003FC0FFE1F0F3C07380336073E0F3EFEB8
:106D5D003FFC3FF03300000BFF3FFF3FFF3F830140
:106D6D0083038307830FC71FFF3DFE387C30000070
:106D7D000B3C0C7E1CFF3CE738C330C330C330C71F
:106D8D0039CF3F8E1F0C0F00000A000003000300D7
:106D9D000300FF3FFF3FFF3F030003000300000020
:106DAD0000000BFF07FF1FFF3F00380030003000D1
:106DBD00300038FF3FFF1FFF0700000B07003F00AB
:106DCD00FF01F80FC03F003EC03FF80FFF013F002D
:106DDD00070000000BFF3FFF3FFF3F001E800780B5
:106DED00038007001EFF3FFF3FFF3F00000B0330F6
:106DFD000F3C1F3E3C0FF003E001F0033C0F1F3E24
:106E0D000F3C033000000B03000F003F00FC00F0AF
:106E1D003FC03FF03FFC003F000F00030000000BA0
:106E2D000330033C033E033FC333E331F3303F30C4
:106E3D001F300F30033000000900000000FF3FFF3E
:106E4D003FFF3F03300330033003300000000000EC
:106E5D00000C0E001E003C007800F000E001C003A5
:106E6D008007000F001E001C001809000000000321
:106E7D0030033003300330FF3FFF3FFF3F00000082
:106E8D000000000C6000700078003C001E000F0038
:106E9D000F001E003C007800700060000C00C00068
:106EAD00C000C000C000C000C000C000C000C000D5
:106EBD00C000C000C00800000000000000003E003F
:106ECD007E007E004E0000000000000000000B0060
:106EDD001C403E603F60336033603360336033E0AD
:106EED003FE03FC03F00000BFF3FFF3FFF3FE03063
:106EFD00603060306030E038E03FC01F800F000030
:106F0D000B800FC01FE03FE03860306030603060B4
:106F1D0030E038C018800800000B800FC01FE03F24
:106F2D00E03860306030E030E030FF3FFF3FFF3F42
:106F3D0000000B800FC01FE03FE03B60336033600B
:106F4D00336033E033C0138001000009C000C0007E
:106F5D00FC3FFE3FFF3FC700C300C300030000001E
:106F6D00000000000B8003C0C7E0CFE0CE60CC6016
:106F7D00CC60CC60EEE0FFE07FE03F00000AFF3F19
:106F8D00FF3FFF3FE00060006000E000E03FC03FDA
:106F9D00803F00000000090000000000306030EC70
:106FAD003FEC3FEC3F0030003000000000000009D6
:106FBD0000000000006000E000E060C0ECFFECFFAE
:106FCD00EC7F0000000000000A0000FF3FFF3FFFC4
:106FDD003F8007C00FE01FE03C603800300000002C
:106FED0000090000000000300330FF3FFF3FFF3F6E
:106FFD00003000300000000000000BE03FE03FE0FB
:10700D003FE000E03FC03FE03FE000E03FC03F8099
:10701D003F00000B0000E03FE03FE03F60006000FC
:10702D006000E000E03FC03F803F00000B800FC0DC
:10703D001FE03FE038603060306030E038E03FC046
:10704D001F800F00000BE0FFE0FFE0FF601C6018E9
:10705D0060186018E01CE01FC00F800700000B8057
:10706D0007C00FE01FE01C601860186018601CE07E
:10707D00FFE0FFE0FF00000B0000E03FE03FE03FDE
:10708D00E000600060006000E000E000C000000073
:10709D0009C011E033E033603360336033603F602B
:1070AD003F401E0000000000000960006000FE1F50
:1070BD00FE3FFE3F60306030603000300000000069
:1070CD0000000BE00FE01FE03F0038003000300003
:1070DD00300038E03FE03FE03F00000B6000E00192
:1070ED00E007801F003E0038003E801FE007E001F2
:1070FD00600000000BE007E01FE03F003CE01FE0F8
:10710D000FE01F003CE03FE01FE00700000A603089
:10711D00E038E03DC01F800F800FC01FE03DE0381C
:10712D006030000000000A00006000E081E0E780B0
:10713D00FF007E801FE007E0016000000000000AF4
:10714D0060306038603C603E6037E033E031E03005
:10715D0060302030000000000A00008000C001FCFB
:10716D001FFE3F7F7F077003600360036000000018
:10717D0000070000000000000000FF3FFF3FFF3F41
:10718D00000000000000000000000A000003600382
:10719D0060036007707F7FFE3FFC1FC00180000011
:1071AD000000000B100018001C000C000C001C004F
:1071BD00180018001C000C00040000000B000F80CC
:1071CD000FC00FE00C700C300C700CE00CC00F8079
:0571DD000F000F00008F
:1071E2001900000000000000000000000000000084
:1071F2000000000000000000000000E001000000AC
:1072020000F00300000000F00300000000F00300A3
:10721200000000F00300000000F00300000000F096
:107222000300000000F00300000000F00300000073
:1072320000F00300000000F00300000000F0030073
:10724200000000F00300000000F00300000000F066
:107252000300000000F00300000000F00300000043
:1072620000F00300000000F00300000000E0010055
:10727200000000C00000000000000000000000004C
:1072820000000000000000000000000000000000FC
:1072920000000000001200000000000000000000DA
:1072A20000000000000000000000000000000000DC
:1072B20000000000000000000000000000000000CC
:1072C20000000000000000000000000000000000BC
:1072D200000000000000000000000000C00F0000DD
:1072E2000000C00F00000000C00F00000000C00F2F
:1072F20000000000C00F00000000C00F00000000EE
:10730200C00F0000000000000000000000000000AC
:10731200000000000000000000000000000000006B
:10732200000000000000000000000000000000005B
:10733200000000000000000000000000000000004B
:10734200000000000000000000001B000000000020
:107352000000000000000300000000C00700000061
:1073620000F00F00000000FC0F00000000FF0F0003
:107372000000C0FF0F000000F0FF0F000000FCFF44
:1073820007000000FFFF01000080FF7F0000008077
:10739200FF1F00000080FF0700000080FF010000C7
:1073A20080FF7F000000E07F00000000F87F000007
:1073B2000000FE7F00000080FF7F000000E0FF1F52
:1073C200000000F8FF07000000FCFF01000000FCC5
:1073D2007F00000000FC1F00000000FC070000000E
:1073E20000F801000000007800000000000000002A
:1073F2000000000000000000000000000000001C6F
:10740200000000000000B0FFFFFF7F00F8FFFFFF59
:10741200FF07FCFFFFFFFF0FFCFFFFFFFF0FFCFF5B
:107422003FFFFF0FFCFF1FFEFF0FFCFF0FFCFF0FD4
:10743200FC000000C00FFC000000C00FFC000000B8
:10744200C00FFC000000C00FFC000000C00FFC00D9
:107452000000C00FFC000000C00FFC000000C00FC5
:10746200FC000000C00FFC000000C00FFC00000088
:10747200C00FFC000000C00FFC000000C00FFCFFAA
:107482000FFCFF0FFCFF1FFEFF0FF8FF3FFFFF0780
:10749200F8FFFFFFFF07F8FFFFFFFF07F8FFFFFFFF
:1074A200FF07F0FFFFFFFF030000000000000000E5
:1074B200000000001C0000000000000000000000AE
:1074C20000000000000000000000000000000000BA
:1074D20000000000000000000000000000000000AA
:1074E200000000000000000000000000000000009A
:1074F200000000000000000000000000000000008A
:107502000000000000000000000000000000000079
:107512000000000000000000000000000000000069
:107522000000000000000000000000000000000059
:10753200000000E0FF0FFCFF01F8FF1FFEFF07FC49
:10754200FF3FFFFF0FFCFFFFFFFF0FFCFFFFFFFFEF
:107552000FF8FFFFFFFF07F0FF3FFFFF03000000F0
:107562000000000000000000001C000000000000FD
:10757200300080FF7F00780080FFFF077C0080FFE3
:10758200FF0F7C00C0FFFF0FFC00E0FFFF0FFC00BD
:10759200F0FFFF0FFC00F0FFFF0FFC00F003C00F35
:1075A200FC00F003C00FFC00F003C00FFC00F0036E
:1075B200C00FFC00F003C00FFC00F003C00FFC0082
:1075C200F003C00FFC00F003C00FFC00F003C00F7B
:1075D200FC00F003C00FFC00F003C00FFC00F0033E
:1075E200C00FFC00F003C00FFCFFFF03C00FFCFF45
:1075F200FF03C00FF8FFFF01C00FF8FFFF00000FED
:10760200F8FF7F000000F8FF7F000000F0FF7F001E
:1076120000000000000000000000000000001C004C
:1076220000000000000000000000003800000080A0
:10763200077C000000800F7C00C000800FFC00E08F
:1076420001C00FFC00F003C00FFC00F003C00FFCF0
:1076520000F003C00FFC00F003C00FFC00F003C0F9
:107662000FFC00F003C00FFC00F003C00FFC00F0A1
:1076720003C00FFC00F003C00FFC00F003C00FFCBE
:1076820000F003C00FFC00F003C00FFC00F003C0C9
:107692000FFC00F003C00FFC00F003C00FFCFFFF63
:1076A200FFFF0FFCFFFFFFFF0FF8FFFFFFFF07F8D1
:1076B200FFFFFFFF07F8FFFFFFFF07F8FFFFFFFFD6
:1076C20007F0FFFFFFFF03000000000000000000C2
:1076D2000000001C000000000000F0FF3F0000005E
:1076E200F0FF7F000000F0FF7F000000E0FFFF00DE
:1076F2000000E0FFFF010000E0FFFF030000C0FF09
:10770200FF0300000000F00300000000F00300008F
:107712000000F00300000000F00300000000F0038E
:1077220000000000F00300000000F0030000000071
:10773200F00300000000F00300000000F00300006E
:107742000000F00300000000F00300000000F0035E
:107752000000E0FFFFFFFF01F8FFFFFFFF07FCFF54
:10776200FFFFFF0FFCFFFFFFFF0FFCFFFFFFFF0FFD
:10777200F8FFFFFFFF07F0FF3FFFFF0300000000DD
:1077820000000000000000001C000000000000B02B
:10779200FF7F000003F8FF7F008007FCFF7F00806F
:1077A2000FFCFFFF00800FFCFFFF01C00FFCFFFF7B
:1077B20003C00FFCFFFF03C00FFC00F003C00FFC6F
:1077C20000F003C00FFC00F003C00FFC00F003C088
:1077D2000FFC00F003C00FFC00F003C00FFC00F030
:1077E20003C00FFC00F003C00FFC00F003C00FFC4D
:1077F20000F003C00FFC00F003C00FFC00F003C058
:107802000FFC00F003C00FFC00F0FFFF0FFC00F0C4
:10781200FFFF0FFC00E0FFFF073C00C0FFFF070077
:107822000080FFFF07000080FFFF07000080FFFFCE
:10783200030000000000000000000000001C000027
:1078420000000000B0FFFFFF7F00F8FFFFFFFF070F
:10785200FCFFFFFFFF0FFCFFFFFFFF0FFCFFFFFF1F
:10786200FF0FFCFFFFFFFF0FFCFFFFFFFF0FFC00FE
:10787200F003C00FFC00F003C00FFC00F003C00FC8
:10788200FC00F003C00FFC00F003C00FFC00F0038B
:10789200C00FFC00F003C00FFC00F003C00FFC009F
:1078A200F003C00FFC00F003C00FFC00F003C00F98
:1078B200FC00F003C00FFC00F003C00FFC00F0FF5F
:1078C200FF0FFC00F0FFFF0FFC00E0FFFF073C0092
:1078D200C0FFFF07000080FFFF07000080FFFF07D7
:1078E200000080FFFF030000000000000000000015
:1078F20000001C000000000000B0FF7F000000F844
:10790200FF7F000000FCFF7F000000FCFF7F000003
:1079120000FCFF3F000000FCFF1F000000FCFF0F07
:10792200000000FC0000000000FC0000000000FC61
:107932000000000000FC0000000000FC000000004D
:1079420000FC0000000000FC0000000000FC000041
:10795200000000FC0000000000FC0000000000FC31
:107962000000000000FC0000000000FC000000001D
:1079720000FCFF0FFCFF01FCFF1FFEFF07F8FF3FAB
:10798200FFFF0FF8FFFFFFFF0FF8FFFFFFFF0FF8EA
:10799200FFFFFFFF07F0FF7FFFFF03000000000073
:1079A200000000000000001C000000000000B0FF0A
:1079B200FFFF7F00F8FFFFFFFF07FCFFFFFFFF0F46
:1079C200FCFFFFFFFF0FFCFFFFFFFF0FFCFFFFFFAE
:1079D200FF0FFCFFFFFFFF0FFC00F003C00FFC00D6
:1079E200F003C00FFC00F003C00FFC00F003C00F57
:1079F200FC00F003C00FFC00F003C00FFC00F0031A
:107A0200C00FFC00F003C00FFC00F003C00FFC002D
:107A1200F003C00FFC00F003C00FFC00F003C00F26
:107A2200FC00F003C00FFCFFFFFFFF0FFCFFFFFF96
:107A3200FF0FF8FFFFFFFF07F8FFFFFFFF07F8FF49
:107A4200FFFFFF07F8FFFFFFFF07F0FFFFFFFF0346
:107A52000000000000000000000000001C00000008
:107A6200000000B0FF7F000003F8FF7F008007FCEA
:107A7200FF7F00800FFCFFFF00800FFCFFFF01C0B3
:107A82000FFCFFFF03C00FFCFFFF03C00FFC00F061
:107A920003C00FFC00F003C00FFC00F003C00FFC9A
:107AA20000F003C00FFC00F003C00FFC00F003C0A5
:107AB2000FFC00F003C00FFC00F003C00FFC00F04D
:107AC20003C00FFC00F003C00FFC00F003C00FFC6A
:107AD20000F003C00FFC00F003C00FFCFFFFFFFF2C
:107AE2000FFCFFFFFFFF0FF8FFFFFFFF07F8FFFF8D
:107AF200FFFF07F8FFFFFFFF07F8FFFFFFFF07F099
:107B0200FFFFFFFF03000000000000000000000074
:017B12000072
:107B13001620201A080C00000000000000000000DE
:107B23000000000000000000000000000000000052
:107B33000000000000000000000000000000000042
:107B43000000000000000000000000000000000032
:107B53000000000000000000000000000000000022
:107B6300000000000000000000000000000007000B
:107B7300000000000000000000000000000000FC06
:107B8300FF010EFCFF3F0EFCFF030E000000000090
:107B930000000000000000000000000000000000E2
:107BA30000000000000000000000000000000000D2
:107BB30000000000000000000000000000000000C2
:107BC300000000000000000B0000000000000000A7
:107BD30000000000FC010000FC070000FC030000A3
:107BE3000000000000000000FC030000FC07000090
:107BF300FC01000000000000000000000000000085
:107C03000000000000000000000000000000000071
:107C13000000000000000000000000000000000061
:107C2300140000000000000000001C0E00001C0EE9
:107C33000E001CFE0F009CFF0F00FCFF01E0FF0F76
:107C430000FC7F0E00FC1F0E001C1C0E00001C0E0F
:107C53000E001CFE0F009CFF0F00FCFF01E0FF0F56
:107C630000FC7F0E00FC1F0E001C1C0E00001C0EEF
:107C730000000000000000000011000000000000F0
:107C8300000000000000C00F7000F01FF001F83F7B
:107C9300F0037878C0073C70000F1C70000EFFFFE4
:107CA300FF7FFFFFFF7F1CE0000E7CE0010FF8C1A8
:107CB3008307F081FF07C001FF010000FE00000001
:107CC30000000000000000000000000000000000B1
:107CD300000016000000000000000000000000C0CB
:107CE3000F0000F03F0000F87F00003CF000001C94
:107CF300E000001CE000001CE0000C3CF0000FF86A
:107D03007FC00FF03FF003C00FFC0000003E0000F7
:107D1300800F0000E0070000F80100007E000080F3
:107D23001FFC00E007FF03F881FF071500000000B8
:107D3300000000000000000000007C000000FE01C5
:107D43000000FF03E083C707F0CF010FF8FF000E29
:107D53003CF8000E1CF0000E1CF0010E1CB8070FBF
:107D63003C1C0F07F81F9E07F00FF803E003F80110
:107D73000000FF0100009F070000020F0000000643
:107D830000000000060000000000000000000000EA
:107D930000FC030000FC070000FC030000000000DF
:107DA30000000000000000000000000000000000D0
:107DB30000000000000000000000000000000000C0
:107DC30000000000000000000000000000000000B0
:107DD300000000000000000000000000000C000094
:107DE300000000000000000000000000000000E0B0
:107DF300FF0000FEFF0F80FFFF3FE01F00FFF801C1
:107E030000F07C0000C01C00000004000000000023
:107E1300000000000000000000000000000000005F
:107E2300000000000000000000000000000000004F
:107E33000000000000000A00000000000000000431
:107E43000000001C0000007C0000C0F80100F0E00E
:107E53001F00FF80FFFF3F00FEFF0F00E0FF000059
:107E6300000000000000000000000000000000000F
:107E730000000000000000000000000000000000FF
:107E83000000000000000000000000000000000DE2
:107E93000000000000000000C0000000E01000002F
:107EA300C0390000801F0000FC0F0000FC0300002D
:107EB300FC0F0000801F0000C0390000E01100002B
:107EC300C0000000000000000000000000000000EF
:107ED300000000000000000000000000000000009F
:107EE300000000000000000014000000000000007B
:107EF30000000000000080030000800300008003F6
:107F03000000800300008003000080030000800362
:107F13000000FEFF0000FEFF0000FEFF00008003E4
:107F23000000800300008003000080030000800342
:107F33000000800300008003000000000000000038
:107F43000007000000000000000000000000000027
:107F530000000000008E000000CE0000007E000044
:107F6300000000000000000000000000000000000E
:107F730000000000000000000000000000000000FE
:107F830000000000000000000000000000000000EE
:107F9300000000000000000000000B0000000000D3
:107FA3000000000000000000000E0000000E0000B2
:107FB300000E0000000E0000000E0000000E000086
:107FC300000E0000000E0000000000000000000092
:107FD300000000000000000000000000000000009E
:107FE300000000000000000000000000000000008E
:107FF3000000000700000000000000000000000077
:10800300000000000000000E0000000E0000000E43
:10801300000000000000000000000000000000005D
:10802300000000000000000000000000000000004D
:10803300000000000000000000000000000000003D
:108043000000000000000000000000000A00000023
:1080530000000000000000800F0000FC0F00C0FFC4
:108063000700FC7F00C0FF0700FC3F0000FC03008B
:10807300003C0000000000000000000000000000C1
:1080830000000000000000000000000000000000ED
:1080930000000000000000000000000000000000DD
:1080A30000000000001100000000000000000000BC
:1080B300000000FE1F00C0FFFF00F0FFFF03F801F8
:1080C300E007380000071C00000E1C00000E1C0017
:1080D300000E1C00000E38000007F801E007F0FF57
:1080E300FF03C0FFFF0000FE1F00000000000000B0
:1080F30000000000000000000000000000000D0070
:10810300000000000000000000000000000000006C
:10811300000000000E00000007000080030000C004
:10812300030000E0010000F8FFFF0FFCFFFF0FFC5E
:10813300FFFF0F000000000000000000000000002F
:10814300000000000000000000000000000000002C
:10815300000000000000001100000000000000000B
:10816300000000008003000EE003800FF003C00F47
:108173007800F00F3C00F80E1C007C0E1C003E0E35
:108183001C001F0E1C800F0E3CC0030E78F0010E66
:10819300F8FF000EE07F000EC00F000E000000008D
:1081A30000000000000000000000000000000000CC
:1081B30012000000000000000000000000800160C9
:1081C30000E001E001F001E003780080073C0000DB
:1081D300071C00000E1C70000E1C70000E1C7000AB
:1081E3000E3C78000F78FC0007F8DFC107F08FFF23
:1081F30003C087FF0100007E0000000000000000B4
:108203000000000000000000001200000000000059
:1082130000000000000000003C0000003F0000C020
:108223003F0000F03B0000FC3800003F3800C00F67
:108233003800F0033800FC003800FCFFFF0FFCFFA0
:10824300FF0FFCFFFF0F00003800000038000000A4
:1082530038000000000000000000000000000000E3
:1082630000001200000000000000000000000000F9
:10827300706000E07FE001FC7FE003FC7F80071C6F
:1082830038000F1C1C000E1C1C000E1C1C000E1CB6
:108293001C000E1C3C000F1C3880071CF8C0071C78
:1082A300F0FF031CE0FF0000803F0000000000001F
:1082B30000000000000000000000001100000000AA
:1082C300000000000000000000FC1F00C0FFFF00D2
:1082D300E0FFFF03F0E0C107787000073C30000EB9
:1082E3001C38000E1C38000E1C38000E3C78000FA2
:1082F30078F0C007F8E1FF03F0C1FF0180017F00C0
:10830300000000000000000000000000000000006A
:108313000000000011000000000000000000000049
:10832300001C0000001C0000001C0000001C00805A
:108333000F1C00F80F1C00FF0F1CE07F001CF80748
:10834300001CFE00009C1F0000DC070000FC000076
:10835300007C0000001C0000000000000000000082
:1083630000000000000000000000000000110000F9
:108373000000000000000000000000007E00C08735
:10838300FF01F0CFFF03F8DF81073CF8000F1C70FB
:10839300000E1C70000E1C70000E1C70000E78F88E
:1083A300000FF8DF8107F0CFFF03C087FF01000054
:1083B3007E0000000000000000000000000000003C
:1083C3000000000000001100000000000000000099
:1083D300000000803FE000E0FFE003F0FFE107F86A
:1083E300E083073C80070F1C00070E1C00070E1CD0
:1083F30000070E1C00030F38808307F8E0E103F049
:10840300FFFF01C0FFFF0000FE0F0000000000009F
:0F8413000000000000000000000000000000005A
:10842200161C201A080C00000000000000000000CA
:10843200000000000000000000000000000000003A
:10844200000000000000000000000000000000002A
:10845200000000000000000000000000000000001A
:10846200000000000000000000000000000000000A
:1084720000000000000000000000000000000500F5
:10848200000000FC7FF000FEFFF803FEFFF803FC93
:108492007FF000000000000000000000000000006B
:1084A20000000000000000000000000000000000CA
:1084B20000000000000000000000000000000000BA
:1084C20000000000000000000000000000000000AA
:1084D200000000000000000C00000000F800000096
:1084E200FE030000FE030000F80000000000000090
:1084F2000000000000000000F8000000FE03000081
:10850200FE030000F8000000000000000000000070
:108512000000000000000000000000000000000059
:108522000000000000000000000000000000000049
:10853200130000000000040200000E0700000E07F6
:1085420000000E0700F0FF7F00F8FFFF00F0FF7F42
:1085520000000E0700000E0700000E0700000E07C5
:1085620000F0FF7F00F8FFFF00F0FF7F00000E0722
:1085720000000E0700000E070000040200000000C9
:108582000000000000000000001300000000C00313
:108592000000E0076000D00FF000B817F00078305C
:1085A200F0007878F0007878F0007878F000FEFF3C
:1085B200FF03FEFFFF03FEFFFF037878F0007878E9
:1085C200F0007830F00078A0EF0078C05F003080D3
:1085D2003F0000801F0000000000000000000000BB
:1085E20000001200000000C000F800E001FC00F0F2
:1085F20003FE00E0037F00C0813F0080C01F000037
:10860200E00F0000F8070000FC030000FE0100007C
:10861200FF0000807F0000C03F3000E01F7800F0C4
:1086220007FC00F0037800F00130000000000000B9
:108632000000000000000000000000100000000028
:1086420000073E00800F7F00C09FFF00E0BFF701E0
:10865200F0FDF30178F8E101F8F8E101F0FDF30132
:10866200E0BFF701C01FFF00800F7E0000077E0001
:108672000080FF000080F7000080E300000000009F
:1086820000000000000000000000000000000000E8
:10869200000000000500000000F8000000FE0300DA
:1086A20000FE030000F800000000000000000000CF
:1086B20000000000000000000000000000000000B8
:1086C20000000000000000000000000000000000A8
:1086D2000000000000000000000000000000000098
:1086E200000000000000000000000000000A00007E
:1086F2000000C0FF1F00E0FF3F00F0FF7F00ECFF23
:10870200BF011E00C0031E00C0031E00C0031E00E6
:10871200C0030C0080010000000000000000000007
:108722000000000000000000000000000000000047
:108732000000000000000000000000000000000037
:108742000000000000000B00000000000000000C10
:108752000080011E00C0031E00C0031E00C0031ED5
:10876200008001E8FFBF00F0FF7F00E0FF3F00C094
:10877200FF1F0000000000000000000000000000D9
:1087820000000000000000000000000000000000E7
:1087920000000000000000000000000000000011C6
:1087A2000000000078207000F8707800F0713C0042
:1087B200E0731E00C0770F0080FF070000FF070074
:1087C20000FE030000FE030000FE070000FF07009A
:1087D200C0770F00E0731E00F0713C00F870780063
:1087E200782070000000000000000000000000007F
:1087F20000000000000000000F0000000000400028
:10880200000060000000F0000000F0000000F00036
:108812000000FF0F0080FF3F0080FF3F0000FF0FBE
:108822000000F0000000F0000000F0000000600016
:1088320000004000000000000000000000000000F6
:108842000000000000000000000000000000000026
:10885200000500000000000080030000C0030000CB
:10886200C0010000C0000000000000000000000085
:1088720000000000000000000000000000000000F6
:1088820000000000000000000000000000000000E6
:1088920000000000000000000000000000000000D6
:1088A200000000000000000000000F0000000000B7
:1088B20060000000F0000000F0000000F000000086
:1088C200F0000000F0000000F0000000F0000000E6
:1088D200F0000000F0000000F0000000F0000000D6
:1088E200F000000060000000000000000000000036
:1088F2000000000000000000000000000000000076
:1089020000000004000080000000C0010000C0035D
:1089120000008000000000000000000000000000D5
:108922000000000000000000000000000000000045
:108932000000000000000000000000000000000035
:108942000000000000000000000000000000000025
:108952000000000000000000000000001200000003
:10896200000000F8000000FC000000FE0000007F94
:108972000000803F0000C01F0000E00F0000F80769
:108982000000FC030000FE010000FF0000807F00E9
:1089920000C03F0000E01F0000F0070000F00300ED
:1089A20000F00100000000000000000000000000D4
:1089B20000000000001300000000F09F7F00F0FFA5
:1089C2007F00F0FF7F00EEFFBF03CE9F9F031E00DC
:1089D200C0031E00C0031E00C0031E00C0031E0011
:1089E200C0031E00C0031E00C0031E00C003CE9FB2
:1089F200DF03E6DFBF03F0FF7F00F0FF7F00F09FA1
:108A02007F000000000000000000000000000A00DB
:108A1200000000080000000C0000001E0000000E14
:108A220000000006000000F207FF00FE8FFF03FEB9
:108A32008FFF03FE07FF000000000000000000009F
:108A42000000000000000000000000000000000024
:108A52000000000000000000000000000000000014
:108A62000000000000000013000000000080FF0072
:108A72000CC0FF001E807F031E60BF031EF0C003F8
:108A82001EF0C0031EF0C0031EF0C0031EF0C003A0
:108A92001EF0C0031EF0C0031EF0C0031EF0C00390
:108AA2000EE0C003E6CFC003F61FC003F83F80010B
:108AB200F83F00000000000000000000000000007D
:108AC2001300000000000000000C6080011EF0C0D6
:108AD200031EF0C0031EF0C0031EF0C0031EF0C050
:108AE200031EF0C0031EF0C0031EF0C0031EF0C040
:108AF200031EF0C0031E60C003CEDF9F03EEDFBF84
:108B020003F6FF7F03F8FFFF00F89FFF000000005D
:108B12000000000000000000001300000000FC073D
:108B22000000FE1F0000FE1F0000FC1F00000040AE
:108B320000000060000000F0000000F0000000F003
:108B4200000000F0000000F0000000F000000060F3
:108B52000000F8DFFF00FCFFFF01FEFFFF03FCFF48
:108B6200FF01F89FFF00000000000000000000006D
:108B720000001300000000FC070000FA0F8001F65D
:108B82001FC003CE27C0031E30C0031E78C0031EC1
:108B920078C0031E78C0031E78C0031E78C0031E6F
:108BA20078C0031E78C0031E78C0031E30C0031EA7
:108BB200809F010CC07F000080FF0000007F00004A
:108BC2000000000000000000000000130000000090
:108BD200F09F7F00F0FF7F00F0FF7F00EEFFBF03FA
:108BE200CEDF9F031E60C0031EF0C0031EF0C00351
:108BF2001EF0C0031EF0C0031EF0C0031EF0C0032F
:108C02001EF0C0031EE0C0031E40BF031EC07F0053
:108C12000C807F0000007F000000000000000000C8
:108C2200000000001300000000000000000C000023
:108C3200001E0000001E0000001E0000001E0000BA
:108C4200001E0000001E0000001E0000001E0000AA
:108C5200001E0000001E0000001E000000DE9FFF3C
:108C620000EEBFFF01F6FFFF03F8BFFF01F89FFF11
:108C720000000000000000000000000000130000DF
:108C82000000F09F7F00F0FF7F00F0FF7F00EEFF0B
:108C9200BF03CEDF9F031E60C0031EF0C0031EF0A1
:108CA200C0031EF0C0031EF0C0031EF0C0031EF07E
:108CB200C0031E60C003CEDF9F03E4DFBF01F0FFED
:108CC2007F00F0FF7F00F09F7F00000000000000A7
:108CD2000000000000001300000000F01F8000F000
:108CE2003FC001F03FC003EE1FC0031E60C0031E61
:108CF200F0C0031EF0C0031EF0C0031EF0C0031E2E
:108D0200F0C0031EF0C0031EF0C0031E60C003CEFD
:108D1200DF9F03E4DFBF01F0FF7F00F0FF7F00F081
:0F8D22009F7F0000000000000000000000000024
:108D31001A232D0D061500000000000000000000A0
:108D4100000004000000000E000000000E00000002
:108D5100001F000000001F000000001F00000000B5
:108D61001F000000001F000000001F000000001F86
:108D7100000000001F000000001F000000001F0095
:108D81000000001F000000001F000000001F000085
:108D910000001F000000000E0000000004000000A1
:108DA10000000000000000000000000000000000C2
:108DB10000000000000000000700000000000000AB
:108DC100008000000000C001000000E0030000007E
:108DD100E003000000C0010000008000000000006E
:108DE1000000000000000000000000000000000082
:108DF1000000000000000000000000000000000072
:108E01000000000000000000000000000000000061
:108E11000000000000000000000000000000000051
:108E21000000000000000000000000000000000041
:108E31000000000000000000000000190000000018
:108E41000000000000000000007E000000007F0024
:108E51000000807F000000C07F000000E07F000074
:108E610000F03F000000F81F000000FC0F000000B0
:108E7100FE03000000FF01000080FF000000C07F32
:108E8100000000E03F000000F01F000000F80F00AC
:108E91000000FC07000000FE03000000FF010000CD
:108EA100C0FF000000C07F000000C03F000000C004
:108EB1001F000000C00F00000000000000001800AB
:108EC100000000000000000000C0FFF17F00C0FFB3
:108ED100FB7F00C0FFFF7F009CFFFB3F033CFFF1D6
:108EE100CF03FC0000E003FC0000F003FC0000F0F5
:108EF10003FC0000F003FC0000F003FC0000F003A1
:108F0100FC0000F003FC0000F003FC0000F003FC97
:108F11000000F003FC0000F003FC0000F0037CFF04
:108F2100F1EF03BCFFFBDF03C0FFFF3F00C0FFFB0E
:108F31007F00C0FFF17F0000000000000000000082
:108F4100000D0000000000000000000020000000F3
:108F51000070000000007800000000FC000000002C
:108F61007C00000000BCFFE0FF00DCFFF1FF01EC32
:108F7100FFFBFF03F0FFFBFF03F0FFF1FF01F0FF39
:108F8100E0FF000000000000000000000000000001
:108F910000000000000000000000000000000000D0
:108FA10000000000000000000000000000000000C0
:108FB10000000000000000000000000000000000B0
:108FC1000000000019000000000000000000003057
:108FD10000F0FF007800F8FF00FC00F83F03FC0000
:108FE100F69F03FC00E7CF03FC80CFE703FC801F63
:108FF100F003FC801FF003FC801FF003FC801FF0D6
:1090010003FC801FF003FC801FF003FC801FF003B2
:10901100FC801FF003FC801FF003FC801FF003FCA9
:10902100801FF0037C7F1FF003BCFF1CF003DCFFFB
:1090310019F003E0FF03F003E0FF03E001E0FF03A9
:10904100C000000000000018000000000000000047
:109051000000300006C00078000FE001FC801FF026
:1090610003FC801FF003FC801FF003FC801FF00352
:10907100FC801FF003FC801FF003FC801FF003FC49
:10908100801FF003FC801FF003FC801FF003FC80B5
:109091001FF003FC801FF003FC801FF003FC801F06
:1090A100F003FC000FF0037CFFF5CF03BCFFFB9F37
:1090B10003CCFFFF3F03E0FFFBFF00E0FFF0FF00F9
:1090C1000000000000000000000018000000000087
:1090D1000000000000F07F000000F8FF000000FC2D
:1090E100FF010000FCFF030000F8FF030000F0FF98
:1090F10005000000000F000000801F000000801F1D
:10910100000000801F000000801F000000801F0081
:109111000000801F000000801F000000801F000071
:1091210000801F000000000F0000F0FFF5FF00F8B5
:10913100FFFBFF01FCFFFFFF03F8FFF9FF01F0FF59
:10914100F0FF000000000000000000000019000016
:109151000000000000000000F83F00C000F47F00A4
:10916100E001ECFF00F003DCFF01F003BCFF06F0BF
:10917100037C7F0FF003FC801FF003FC801FF003D2
:10918100FC801FF003FC801FF003FC801FF003FC38
:10919100801FF003FC801FF003FC801FF003FC80A4
:1091A1001FF003FC801FF003FC000FF003FC00F62E
:1091B100EF03FC00F8DF03FC00FCBF017800F87F3F
:1091C100003000F07F000000E03F000000000000E0
:1091D1001900000000000000000000C0FFF17F0046
:1091E100C0FFFB7F00C0FFFF7F009CFFFB3F033CF4
:1091F100FFF4CF03FC000FE003FC800FF003FC80C1
:109201001FF003FC801FF003FC801FF003FC801F94
:10921100F003FC801FF003FC801FF003FC801FF0B3
:1092210003FC801FF003FC801FF003FC801FF00390
:10923100FC00CEEF03FC00E4DF03FC00F03F00FC88
:1092410000F07F007800E07F002000C07F00000078
:1092510000000018000000000000000000003000C5
:109261000000007800000000FC00000000FC00008D
:109271000000FC00000000FC00000000FC000000F9
:1092810000FC00000000FC00000000FC00000000E9
:10929100FC00000000FC00000000FC00000000FCDD
:1092A10000000000FC00000000FC00000000FC00C9
:1092B1000000007CFEE1FF00BCFFFBFF01DCFFFFC3
:1092C100FF03E0FFFBFF01E0FFE1FF000000000002
:1092D1000000000000001800000000000000000075
:1092E10000C0FFF17F00C0FFFB7F00C0FFFF7F00D8
:1092F10090FFFB3F0138FFF4CF01FC000FE003FCBE
:10930100801FF003FC801FF003FC801FF003FC8032
:109311001FF003FC801FF003FC801FF003FC801F83
:10932100F003FC801FF003FC801FF003FC801FF0A2
:1093310003FC000FF0037CFFF5EF03B8FFFBDF0137
:10934100C0FFFF3F00C0FFFB7F00C0FFF07F0000B8
:1093510000000000000000000018000000000000F4
:1093610000000000C0FF01C000C0FF03E001C0FF1A
:1093710007F003D0FF03F003B8FF05F0037CFF06FD
:10938100F003FC000FF003FC801FF003FC801FF0D2
:1093910003FC801FF003FC801FF003FC801FF0031F
:1093A100FC801FF003FC801FF003FC801FF003FC16
:1093B100801FF003FC000FF0037CFFF5EF03B8FF03
:1093C100FBDF01C0FFFF3F00C0FFFB7F00C0FFF0DC
:0C93D1007F000000000000000000000011
:1093DD001017201A0B09000000000000000000000B
:1093ED000000000000000000000000000000000070
:1093FD000000000000000000000000000000000060
:10940D000000000000000700000000000000000048
:10941D00FE0F0CFEFF1EFE0F1E00000C00000000D4
:10942D00000000000000000000000000000000002F
:10943D0000000000000000090000007E00007E001A
:10944D00007E00000000000000007E00007E000095
:10945D007E00000000000000000000000000000081
:10946D0000000000000000001000000000E01800E7
:10947D00E01FC0F91FC0FF07F0FF00FCE700FCE193
:10948D0018CCE11FC0F91FC0FF07F0FF00FCE7007B
:10949D00FCE100CC0100C001000D00000000000047
:1094AD00E00108F8071EF8071C3C0F1C1F0E3C1F9F
:1094BD001C3C1F3C3C1C781E3CF80F18F00F00C0E4
:1094CD000300000000000000000010F00300F8078A
:1094DD0010FC0F181C0E1C1C0E0F1C8E07FCCF034E
:1094ED00F8F700F07B00003E0000EF0780F70FE07B
:1094FD00F91FF0381C78381C1C381C10000000F0C7
:10950D00E103F8FB07FCFF0F1E1F1E0E0E1C0E0EB7
:10951D001C0E0E1C0E0E1C0E0E1C84FF1F80FF0F4A
:10952D00C0FF1F000E1C000E1C000E1C05000000CD
:10953D000000007E00007E00007E000000000000A4
:10954D00000000000000000000000000000000000E
:10955D0000000000000000000000000000090000F5
:10956D000000000000000000FC0380FF1FE0FF3F33
:10957D00F801301C00000E0000000000000000008B
:10958D0000000000000000000000000000000800C6
:10959D0000000000000E00001C0000F80130E0FF8C
:1095AD003F80FF1F00FC03000000000000000000D2
:1095BD000000000000000000000000000000000B93
:1095CD00200000380100F80300F00700FE0300FE44
:1095DD000000FE0300F00700B80300380300300060
:1095ED00000000000000000000000000000000006E
:1095FD000F000000000000003800003800003800A7
:10960D00003800003800C0FF07C0FF07C0FF07008B
:10961D003800003800003800003800003800000025
:10962D00000700000000000000000000000C00001A
:10963D003E00003E00003C00000000000000000065
:10964D00000000000000000000000000000000000D
:10965D0000000B00000000700000700000700000A2
:10966D00700000700000700000700000700000704D
:10967D00000070000000000000000000000000006D
:10968D000000000700000000000C00001E00003369
:10969D0000003300001E00000C0000000000000060
:1096AD0000000000000000000000000000000000AD
:1096BD00000000000A00001000001E00C01F00F88E
:1096CD000F00FE01C07F00F80F00FC01007C0000C0
:1096DD000C00000000000000000000000000000071
:1096ED0000000000000E00000080FF00E0FF03F00E
:1096FD00FF0F78000F3C001E1C001C1C001C1C00E2
:10970D001C3C001E78000FF8FF07F0FF0380FF00E0
:10971D000000000000000B00000000000000000031
:10972D00000000800300C00100E00100F00000F81F
:10973D00FF1FFCFF1FFCFF1F0000000000000000CA
:10974D00000000000000000F0000000000003000CD
:10975D001878001C38001E3C001F1CC01F1CE01D8B
:10976D001CF01C1C781C3C3E1CF80F1CF8071CE060
:10977D00011C00001C0000000E0000000000000095
:10978D00000000000418000E38001E3C001C1C0ECA
:10979D001C1C0E1C3C0F1CFC1F1EF8FB0FF0F107D0
:1097AD0000E0030000000000000F00000000E000DA
:1097BD0000F00000F80000FC0000FE0080EF00C08B
:1097CD00E700E0E300F0E100F8FF1FFCFF1FFCFFE6
:1097DD001F00E00000E0000000000E00000000008F
:1097ED0000000006FC0F0FFC1F1EFC0F1C1C071CAD
:1097FD001C071C1C071C1C071E1C0F0E1CFE0F1C1F
:10980D00FC0700F8010000000000000E0000000041
:10981D00000000FC0100FF07C0FF0FE01F0EF00E5F
:10982D001C780E1C3C0E1C1C0E1C081E1E00FC0F72
:10983D0000F80700F0030000000000000F0000001A
:10984D000000000000001C00001C00181C001E1C65
:10985D00C01F1CF00F1CFC011C7F00DC0F00FC0363
:10986D0000FC00003C00000C00000000000E000099
:10987D000000000000E003F0F10FF8FB0FF83F1EB1
:10988D001C1F1C1C0E1C1C0E1C3C1F1CFC3F1EF820
:10989D00FB0FF0F10700C0030000000000000E00F8
:1098AD000000000000E00700F00F00F81F003C3C36
:1098BD00081C381C1C381E1C380F1CB80F38FC0730
:0F98CD00F8FF01F0FF00C01F00000000000000C6
:1098DC00050B2060200300000000000000000000C9
:1098EC0003000000007E03000000000400000F00D5
:1098FC0000000F000000054800FE014800FE014872
:10990C00000418012602440688010000040603E640
:10991C000018030603000005DC0122025C02800132
:10992C00400204000000000B0007000000030000D0
:10993C00FC010202000000000300000202FC010016
:10994C000000000548003000FC00300048000520F5
:10995C00002000F800200020000300000003000796
:10996C000000000004200020002000200000000364
:10997C0000000003000300000000040003E00018D6
:10998C00000600000004FC0302020202FE010000BB
:10999C000408020402FE0300020000048C034202CD
:1099AC0022021C02000004040122022202DC01003B
:1099BC000004600058004400FE030000043E012235
:1099CC00022202C201000004F80114021202E20198
:1099DC000000040200820362001E00000004DC018F
:1099EC0022022202DC010000043C0242024201FC81
:1099FC0000000003000030033003000000000300EF
:109A0C0000300330070000000004600090000801E3
:109A1C000402000004A000A000A000A000000004AC
:109A2C0004020801900060000000040C00020062B7
:109A3C00031C00000004FC01020262027C02000014
:109A4C0004FC0322002200FC03000004FE0322029B
:109A5C002202DC01000004FC01020202020C0100E3
:109A6C000004FE0302020202FC01000004FE0322B9
:109A7C000222022202000004FE0322002200220025
:109A8C00000004FC0102024202CC01000004FE03AF
:109A9C0020002000FE0300000400000202FE03026E
:109AAC000200000480010202FE010200000004FE1C
:109ABC00032000D8000603000004FE03000200028D
:109ACC000002000004FE0318001800FE030000044E
:109ADC00FE0318006000FE03000004FC01020202F9
:109AEC0002FC01000004FE03220022001C00000006
:109AFC0004FC0102020206FC01000004FE036200E9
:109B0C00A2001C030000049C0122022202CC0100D2
:109B1C00000502000200FE030200020004FE010028
:109B2C00020002FE010000043E00C0000003FE0023
:109B3C00000004FE0380008000FE030000048E037E
:109B4C00700070008E030000050E003000C0033062
:109B5C00000E0004820362021A02060200000300D7
:109B6C0000FE030202000000000406001800E000E2
:109B7C00000300000300000202FE030000000004CA
:109B8C0000000400020004000000010000000000BE
:109B9C00000000000003000007000B0000000000A4
:109BAC0004800150025002E003000004FE03100286
:109BBC001002E001000004E001100210021002008B
:109BCC000004E00110021002FE03000004E001900A
:109BDC00029002E0020000031000FC0312000000DF
:109BEC00000004E00110021002F007000004FE0364
:109BFC0010001000E00300000400000002F4030059
:109C0C000200000300040000F4070000000004FE42
:109C1C0003C0002001100200000400000202FE0339
:109C2C000002000004F00320002000F003000004F8
:109C3C00F00320001000E003000004E0011002100B
:109C4C0002E001000004F00710021002E001000025
:109C5C0004E00110021002F0070000041000E00301
:109C6C00100030000000042001500290022001007E
:109C7C0000031000FC0310020000000004F00100BF
:109C8C00020002F0030000043000C0000003F000EA
:109C9C00000004F00300010001F003000004300395
:109CAC00C000C0003003000004F00100020002F00C
:109CBC000700000410039002500230020000032041
:109CCC0000DC010202000000000300000000EF03B2
:109CDC00000000000400000202DC0120000000046F
:109CEC000400020004000200000005E00318020654
:059CFC00021802E00364
:109D01000D15201A100700000000000000000000DF
:109D11000000000000000000000000000000000042
:109D2100000000000000000000000000000400002E
:109D310000000000FCDF01FCDF010000000000006A
:109D41000000000000000000000000000000000012
:109D51000000000000070000003C00003C00000083
:109D610000000000003C00003C000000000000007A
:109D7100000000000000000000000000000B0000D7
:109D810000009001407800401700F010004C900155
:109D9100407000401F00F010004C10004000000017
:109DA10000000000000A000000000000F08000F840
:109DB100C1019C83010F83070F86070CC6011CFCA0
:109DC100000078000000000000000000000C00000E
:109DD10000F8000104C100046100041900F8060044
:109DE100000300C0F800300401180401040401005C
:109DF100F8000000000D000000F07E00F8FF001CDC
:109E0100C3010C83010C83010C83011C8301C8FF76
:109E110000E0FF01008301008301008300030000D3
:109E2100003C00003C0000000000000000000000B9
:109E31000000000000000000000000000000000021
:109E4100000000000007000000000000000000000A
:109E51007F00E0FF0338000E0C0018000000000036
:109E610000000000000000000000000000060000EB
:109E7100000000000C001838000EE0FF03007F0016
:109E810000000000000000000000000000000000D1
:109E9100000000000007000000100000D000007C5E
:109EA10000007C0000D00000100000000000000055
:109EB100000000000000000000000000000A000691
:109EC10000000600000600000600E07F00E07F00C1
:109ED1000006000006000006000006000000000069
:109EE100000000000006000000000000000010005B
:109EF100C00800C00700C00300000000000000000F
:109F0100000000000000000000000000000600004A
:109F110000000000000C00000C00000C00000C0010
:109F21000000000000000000000000000000000030
:109F310000000000000500000000000000C001005A
:109F4100C00100C00100000000000000000000008E
:109F510000000000000000000000000000090000F7
:109F61000000000000800100F00100FE00C01F00A1
:109F7100F803007C00000C0000000000000000005D
:109F810000000000000A000000C03F00F0FF0038A0
:109F9100E0010C80010C80010C80011CE000F8FF45
:109FA10000E01F00000000000000000000070000AA
:109FB10000000000600000300000380000F8FF01E0
:109FC100FCFF010000000000000000000000000094
:109FD10000000000000A00000010000118C0010C80
:109FE100E0010CB8010C9C011C8701F88301F08091
:109FF100010080010000000000000000000A0000D4
:10A00100000880001CC0010C80010C83010C83013D
:10A011009C8301F8C60170FE00007C000000000076
:10A0210000000000000B001800001C00001E0000D2
:10A031001B00C01900E01800701800F8FF01FCFFB8
:10A04100010018000018000000000000000A0000D4
:10A0510000000000FC8300FCC1018C81018C8101A6
:10A061008C81018CC3010CFF00007E000000000008
:10A0710000000000000A000000003F00C0FF00E0F7
:10A08100C6017883011883010C830104C70100FE16
:10A0910000007C000000000000000000000B000038
:10A0A100000000000C00000C80010CF0010C7C0091
:10A0B1008C1F00EC0300FC00003C00000C000000C1
:10A0C10000000000000A000000007800F0FE00F827
:10A0D100C7018C83010C83018C8301F8C70170FCDB
:10A0E100000078000000000000000000000A0000ED
:10A0F10000F00100F803001C07010C86010CC600EA
:10A101000CF6001C3B00F81F00E0070000000000F7
:05A11100000000000049
:10A116000608206019040000000000000500000683
:10A126005F0600060007030007030600247E247E60
:10A13600240500242B6A12000600631308646306D4
:10A1460000364956205004000007030000040000B2
:10A156003E410000040000413E00000600083E1C8F
:10A166003E08060008083E0808040000E0600000FB
:10A1760006000808080808040000606000000600E1
:10A18600201008040206003E5149453E05000042E3
:10A196007F40000600625149494606002249494966
:10A1A6003606001814127F1006002F494949310659
:10A1B600003C4A494930060001710905030600368C
:10A1C600494949360600064949291E0400006C6CB7
:10A1D6000000040000EC6C00000500081422410099
:10A1E6000600242424242406000041221408060024
:10A1F600020159090606003E415D551E06007E1104
:10A2060011117E06007F4949493606003E4141410B
:10A216002206007F4141413E06007F4949494106E9
:10A22600007F0909090106003E4149497A06007F77
:10A236000808087F050000417F41000600304040C5
:10A24600403F06007F0814224106007F4040404000
:10A2560006007F0204027F06007F0204087F0600D4
:10A266003E4141413E06007F0909090606003E417E
:10A2760051215E06007F09091966060026494949EB
:10A2860032060001017F010106003F4040403F06C3
:10A29600001F2040201F06003F403C403F06006351
:10A2A600140814630600070870080705007149457D
:10A2B60043000500007F414100060002040810200B
:10A2C60005000041417F00060004020102040680E9
:10A2D6008080808080040000030700000600205470
:10A2E60054547806007F44444438060038444444B5
:10A2F600280600384444447F060038545454080560
:10A3060000087E090900060018A4A4A47C05007FA5
:10A3160004047800050000007D40000500408084AC
:10A326007D0005007F10284400050000007F4000E6
:10A3360006007C0418047805007C040478000600F6
:10A3460038444444380600FC444444380600384443
:10A356004444FC0600447844040806000854545457
:10A36600200500043E44240005003C40207C0006F5
:10A37600001C2040201C06003C6030603C05006C40
:10A3860010106C0005009CA0603C0005006454544D
:10A396004C000500083E4141000400000077000023
:10A3A60006000041413E08050002010201000600C8
:05A3B6003C2623263CBB
:10A3BB00536F75726365203A205F31384632364BE6
:10A3CB0032325F5350495F4C43445F494C493932F9
:10A3DB0032355F445331384232305F5F3138303180
:07A3EB0031392E630D0A0059
:10A3F2004469726563746F7279203A205F4C4344FA
:10A402005F726F7567655F322D32505F3137367814
:10A412003232305F5350495F494C49393232350D3F
:02A422000A002E
:10A424004D65737572652074656D706572617475C0
:10A434007265207669612053656E736F72204F5781
:0FA44400532044533138423230203A200D0A0061
:10A45300466F6E7423332044726177746578742079
:10A4630030313233343536373839303132333435AD
:0EA473002E203120617420312C37300D0A006C
:10A4810050726F6A6574203A2031384632366B3229
:10A49100325F546573745F4C43445F526F756765F7
:0DA4A1005F5350492E6D637070690D0A0005
:10A4AE00416C6C6F636174696F6E2064652033302C
:10A4BE00343520627974657320706F7572206C6507
:0CA4CE007320666F6E7473200D0A20006E
:10A4DA005F4C43445F726F7567655F322D32505F20
:10A4EA00313736783232305F5350495F494C4939F7
:04A4FA0032323500C5
:10A4FE005F31384632364B32325F5350495F4C43F0
:10A50E00445F494C49393232355F44533138423217
:03A51E00305F00AB
:10A5210031384632366B32325F546573745F4C4357
:10A53100445F526F7567655F5350492E6D6370704C
:02A541006900AF
:10A5430044726177746578742041424344454647B9
:10A5530048494A4B4C4D4E20617420312C31360D05
:02A563000A00EC
:10A56500566572746963616C6520206A61756E65F4
:10A57500207669612044726177506978656C200D99
:02A585000A00CA
:10A5870052656374616E676C6520426C616E63200F
:10A59700766961204472617720506978656C0D0A8D
:01A5A70000B3
:10A5A800486F72697A6F6E74616C6520726F756737
:10A5B800652076696120447261774C696E650D0A81
:01A5C8000092
:10A5C900566572746963616C6520204272756E20EC
:10A5D90076696120447261774C696E65200D0A00C5
:10A5E900456372697420656E20583D3020593D34A9
:0FA5F900302020466F6E742334203578313100C6
:10A60800496E697420544654204C434420322C32FD
:0EA6180022203137367832323020200D0A00F1
:10A626004142434445464748494A4B4C4D4E4F509C
:0BA636005152535455565758595A00C2
:10A64100506F77657220737570706C793A20332E74
:0AA651003320746F2035560D0A0007
:10A65B00447261772020466F6E742336202061741C
:0AA66B0020312C203134340D0A0098
:10A67500447261772020466F6E7423352020617403
:0AA6850020312C203134300D0A0082
:10A68F003132333435363738393031323334353679
:0AA69F0037383930313233343500DA
:10A6A9004D6178204672656520626C6F63206D6527
:09A6B9006D6F697265203D2000FF
:10A6C200447261772020466F6E74233420206174B7
:09A6D20020312C2033300D0A0068
:10A6DB004C434420313736783232302036354B20DC
:09A6EB00636F756C6575727300F4
:10A6F400447261772020466F6E7423382020617481
:09A7040020312C2039350D0A002A
:10A70D00447261772020466F6E7423372020617468
:09A71D0020312C2034300D0A001B
:10A72600447261772074657874657320736D616C0B
:08A736006C203678380D0A0092
:10A73E0052656374616E676C6520706C65696E201E
:08A74E004A61756E650D0A00F9
:10A75600536576656E5365674E756D466F6E745FAD
:08A766003332783530203D004C
:10A76E00536576656E5365674E756D466F6E745F95
:08A77E0033327835300D0A007A
:10A78600447261772020466F6E74233620206174F0
:08A7960020312C203134350084
:10A79E00506F77657220737570706C793A20332E16
:08A7AE003320746F20355600C2
:10A7B600496E6974204D656D6F7279204D616E61C9
:07A7C600676572200D0A0017
:10A7CD00447261772020466F6E74233720206174A8
:07A7DD0020312C2034300074
:10A7E40052656374616E676C6520706C65696E2078
:07A7F4004359414E0D0A001C
:10A7FB00447261772020466F6E7423382020617479
:07A80B0020312C2038300041
:10A812004C6962657265206C61206D656D6F69724D
:06A822006520320D0A0062
:10A828004469676974616C5F375F4D6F6E6F333071
:06A83800783436203D00DB
:10A83E0046696E207061727469652047726166693F
:06A84E007175650D0A00A2
:10A854004469676974616C5F375F4D6F6E6F333045
:06A864007834360D0A00F5
:10A86A0020464F534320696E7465726E65203A2004
:06A87A0033324D487A0064
:10A88000417269616C5F4E6172726F7732327833F8
:05A8900032200D0A005A
:10A895005472656275636865745F4D5331367832FD
:05A8A50033200D0A0044
:10A8AA00417269616C5F4E6172726F7732327833CE
:05A8BA0032203D2000EA
:10A8BF0045727265757220636C6F736520666F6E7B
:05A8CF0074200D0A00D9
:10A8D400436572636C6520506C65696E20474F4C0C
:04A8E400440D0A0015
:10A8E8005472656275636865745F4D5331337832AD
:04A8F800313D2000CE
:10A8FC005472656275636865745F4D533136783296
:04A90C00333D2000B7
:10A910005472656275636865745F4D533133783284
:04A92000310D0A00EB
:10A92400506172746965204772616669717565204A
:03A934000D0A0009
:10A9370053656E736F72204F57532044533138421B
:03A94700323000AB
:10A94A007061756C666A756A6F2E667265652E66C9
:02A95A00720089
:10A95C0052656374616E676C6520426C616E630D49
:02A96C000A00DF
:10A96E00303132333435363738393031323334359D
:02A97E002E00A9
:10A98000546F74616C2052414D2046726565203DC4
:02A990002000A5
:10A99200205465726D696E616C35783131200D0A13
:01A9A20000B4
:10A9A300447261774C696E6520426C6575650D0A6A
:01A9B30000A3
:10A9B40054656D7020445331384232302023313D88
:01A9C4000092
:10A9C500447261774C696E652056657274650D0A2F
:01A9D5000081
:10A9D600202063666F6E742E6E62726F77733D20F1
:01A9E6000070
:10A9E700202063666F6E742E6865696768743D2002
:01A9F700005F
:10A9F800436572636C65204D4147454E54410D0ACD
:01AA0800004D
:10AA090054656D7020445331384232302023313D32
:01AA1900003C
:10AA1A0020464F534320203A2033324D487A0D0ABC
:01AA2A00002B
:10AA2B005465726D696E614C3132783136203D2040
:01AA3B00001A
:10AA3C0056657273696F6E203A2031383031313976
:01AA4C000009
:10AA4D004D4355203A2031384632364B32320D0ABD
:01AA5D0000F8
:10AA5E00436572636C65204D6172726F6E0D0A00F4
:10AA6E00204E49375345473232783238203D200048
:10AA7E002E2E45727265757220212121200D0A003D
:10AA8E005465726D696E614C31327831360D0A0043
:10AA9E0050617274696520477261666971756500EF
:0FAAAE004142434445464748494A4B4C4D4E00B0
:0FAABD004D4355203A2031384632364B32320065
:0FAACC00436572636C65204A61756E650D0A0003
:0FAADB005465726D696E614C367838203D2000ED
:0FAAEA004E49375345473232783238200D0A0033
:0FAAF9005465726D696E616C35783131203D00A6
:0FAB0800202063666F6E742E4D6178433D2000F0
:0EAB1700205461696C6C6520466F6E742000DE
:0EAB25004E49375345473236783335203D00D0
:0EAB33004E493753454732367833350D0A0008
:0EAB410054656D7020445331384232303D006F
:0EAB4F00496E6974202053504931200D0A00D0
:0EAB5D005465726D696E614C3678380D0A00D1
:0EAB6B0063666F6E742E77696474683D200017
:0EAB7900436572636C6520566572740D0A00A8
:0DAB870050726573656E746174696F6E00C5
:0DAB940020436C6F736520466F6E742000C7
:0CABA1004D696B726F4320372E3130007D
:0CABAD00436C656172205446540D0A0090
:09ABB9000D0A52656375203A0093
:08ABC2002020202020202000AB
:08ABCA002020202020202000A3
:08ABD20020202020202020009B
:07ABDA00206D6178593D0078
:06ABE100B043200D0A0044
:06ABE700B043200D0A003E
:06ABED00B043200D0A0038
:06ABF3006D6178583D0081
:01ABF900005B
:01ABFA000159
:01ABFB000F4A
:020000040030CA
:0D000100381F3CFFBF81FF0FC00FE00F4014
:0200000400F00A
:1000000031384632364B32322054657374204932CF
:1000100043204C43442034783230206361720D0019
:10002000554152542031392C3220382C4E2C312D50
:10003000426C7565546F6F746820484330360D000C
:100040005254432044533133303720656E204932B7
:1000500043202020466F73633D31364D487A0D00B2
:100060007265762031342D30352D323031342020F8
:100070004D696B726F4320202056362E30310D00B3
:10008000496E6974204932432062757320343030E0
:100090004B487A2000496E697420525443204453DF
:1000A00031333037202020202000496E69742041F0
:1000B000444320302D3556205241302D3100FFFF72
:1000C000FFFFFFFFFFFFFFFFFFFFFFFFFFFFFFFF40
:1000D000FFFFFFFFFFFFFFFFFFFFFFFFFFFFFFFF30
:1000E000FFFFFFFFFFFFFFFFFFFFFFFFFFFFFFFF20
:1000F000FFFFFFFFFFFFFFFFFFFFFFFFFFFFFFFF10
:00000001FF
